:03000000020253A6
:03000300D2C12245
:05000600D2C0D2C122AE
:03000B0002522D71
:10000E00E5F06010C3EC13FCED13FDEE13FEEF13E1
:05001E00FFD5F0F02207
:030023000292B690
:10002600CD30E11520E00FC083C08288828C83CD5D
:0C003600F0D082D08322CDF222CDF62241
:10004200CB30E11520E00FC083C08289828A83CB46
:0C005200F0D082D08322CBF322CBF72227
:10005E00ED30E11320E00EC083C08288828C83E0F5
:10006E00D082D08322E2226405700EC083C08288C3
:0B007E00828C8393D082D08322E62284
:1000890088F0A8817404C0E0C0F018E6C0E008E672
:10009900C0E00886F018188001A3E0C608D5F0F979
:0200A900F8223B
:1000AB00EEC0E0EFC0E088F0E58124FDF8ECC6C0BF
:0900BB00E008EDC6C0E0A8F02247
:0C00C400E0A3FCE0A3FDE0A3FEE0FF22AF
:0C00D000ECF0A3EDF0A3EEF0A3EFF022A3
:0C00DC00E208FCE208FDE208FEE2FF2260
:0C00E800E309FCE309FDE309FEE3FF224D
:0C00F400ECF309EDF309EEF309EFF32241
:1001000075F004AA83AB82D083D082E493A3CAC5DE
:1001100083CACBC582CBF0A3CAC583CACBC582CB69
:08012000D5F0E8C082C0832283
:10012800120231C380021819E637F6DAF902022200
:10013800E0A3FEE0FFEF8DF0A4CFC5F0CCA42CFC2B
:09014800EE60038DF0A42CFE22F0
:10015100C2D1C2D5EE30E707D2D1D2D51201FEEC21
:1001610030E705B2D112020612017930D103120132
:10017100FE30D50312020622BC000EBE0032EF8D06
:10018100F08420D226FFADF0227B0075F008EF2F1E
:10019100FFEE33FEEB33FBEE9DEB9C4005FBEE9D4A
:1001A100FE0FD5F0E9E4CECDCBCC227EFF7FFF223E
:1001B100EDB410005022EE8DF084FEEF54F045F0C6
:1001C100C48DF084C4FCEF540FC445F0C48DF08499
:1001D100FFADF0E4CC4FFF22EE8DF08420D2CC7E37
:1001E10008CEC5F0CDCBEF2FFFED33FD10D7079B28
:1001F1005005D5F0F1229BFD0FD5F0EA22C3E49F13
:0D020100FFE49EFE22C3E49DFDE49CFC2270
:0C020E00EE30E707E4C39FFFE49EFE22F1
:10021A0074F9800674FA800274FCD083D082258136
:07022A00F581C082C08322B0
:0F023100E5D054182407F8E58124FCF97A04225B
:10024000EFB40A077F0D1202407F0A3099FDC29970
:030250008F992261
:0F025300758122E4787FF6D8FD75A0000257DB95
:0702620075850175C01B2228
:03026900C2C022EE
:05026C00C2C0D2C22255
:0A027100C20874017900F31207F5CA
:10027B00129201EF7901F3E314600B14601F146009
:06028B0040146053805492
:100291007900E3B40101D340077900E314F380440A
:0D02A10074067900F3803D7900E3B4060691
:0602AE001207F5E4FF2237
:1002B4007900E3FF121EA8EF7802F2E2B404037F90
:1002C400042230081CE4FF227900E3B4060050073E
:1002D4007900E304F3800A74017900F380037F0456
:1002E400227900E3B4040302044E5013E3146020A3
:1002F4001470030203A6147003020409020676E3D1
:1003040024FB700302049314700302050D02027BA4
:100314007B027A0079E17D057C15786912081D7FDE
:10032400017B027A0079E11291389000DEE0700BD3
:100334007F027B057A15797A1291389000DEE0FA13
:10034400B4010B7F027B057A15798B1291389000EA
:10035400DEE0FAB4020B7F027B057A15799C1291D8
:10036400389000DEE0FAB4030B7F027B057A15793E
:10037400AD1291389000DEE0FAB4040B7F027B05E5
:100384007A1579BD1291389000DEE0FAB405028046
:10039400030206767F027B057A1579CE1291380224
:1003A400027B7B027A0079E17D057C1578DF1208F7
:1003B4001D7F017B027A0079E11291389000D5E02B
:1003C400600790010CE0B401117B027A0079E17DB1
:1003D400057C1578F012081D801D9000D5E0FDE421
:1003E400C0E0C0057B027A0079E17D057C167801C6
:1003F40012081D158115817F027B027A0079E112B2
:10040400913802027B7B027A0079E17D057C1678C3
:100414001312081D7F017B027A0079E11291389052
:1004240000D3E0C0E0A3E0C0E07B027A0079E17D84
:10043400057C16782412081D158115817F027B0224
:100444007A0079E112913802027B7B027A0079E129
:100454007D057C16783412081D7F017B027A0079B1
:10046400E11291389000DAE0C0E0A3E0C0E07B0242
:100474007A0079E17D057C16784512081D158115F1
:10048400817F027B027A0079E112913802027B902B
:1004940000DEE0FA6402600EEA64036009EA6404C0
:0604A4006004EAB4051E2D
:1004AA007901E3B401057900E314F37901E3B403B4
:1004BA000280030206767900E304F302027B7B02E0
:1004CA007A0079E17D057C16785512081D7F017B3B
:1004DA00027A0079E11291389000DCE0C0E0A3E0F2
:1004EA00C0E07B027A0079E17D057C167845120826
:1004FA001D158115817F027B027A0079E1129138FC
:10050A0002027B7B027A0079E17D057C167866120D
:10051A00081D7F017B027A0079E11291389000DE92
:10052A00E0B403030205D3500CE0601A14604314CC
:10053A00606C020652E024FC70030205FE1470038C
:06054A0002062902065220
:100550009000D3E0C0E0A3E0C0E09000D5E0FDE46F
:10056000C0E0C0057B027A0079E17D057C167877D2
:1005700012081D74FC2581F5810206529000D3E01B
:10058000C0E0A3E0C0E09000D5E0FDE4C0E0C0051D
:100590007B027A0079E17D057C16788812081D744B
:1005A000FC2581F5810206529000D3E0C0E0A3E073
:1005B000C0E09000D5E0FDE4C0E0C0057B027A0019
:1005C00079E17D057C16789912081D74FC2581F56A
:1005D00081807F9000D3E0C0E0A3E0C0E09000D530
:1005E000E0FDE4C0E0C0057B027A0079E17D057C96
:1005F0001678AB12081D74FC2581F581805490009B
:10060000D3E0C0E0A3E0C0E09000D5E0FDE4C0E0AE
:10061000C0057B027A0079E17D057C1678BD120861
:100620001D74FC2581F58180299000D3E0C0E0A3F2
:10063000E0C0E09000D5E0FDE4C0E0C0057B027AB8
:100640000079E17D057C1678CF12081D74FC2581A8
:0F065000F5819000D5E0600790010CE0B4010C3B
:10065F0074209000E6F074419000E7F07F027B0277
:0A066F007A0079E112913802027B53
:080679007401791CF31207F56E
:10068100129201EF791DF3E31460121460271470C4
:0D0691000302071614700302072C02072F46
:10069E00791CE3B40101D34008791CE314F302077B
:0E06AE002F7405791CF38079791CE3B40506DE
:0606BC001207F5E4FF2225
:0706C200900115E0B40118DE
:1006C900791CE3FF122882EF781EF2E2B404037F5B
:0806D9000422300836E4FF2280
:1006E1001207F57F017B057A1A79201291387F0272
:1006F1007B057A1A79311291381291EEE4FE7FFA74
:100701001291D61291EE7E077FD01291D61207F583
:10071100E4FF228019791CE3B405005007791CE33A
:1007210004F3800A7401791CF380037F0422791C8D
:10073100E314600E14601C14602A146038146046BF
:020741008053E3
:100743007B027A0079E17D057C1A784212081D80CC
:10075300427B027A0079E17D057C1A785312081DE9
:1007630080317B027A0079E17D057C1A7864120876
:100773001D80207B027A0079E17D057C1A78751251
:10078300081D800F7B027A0079E17D057C1A78864B
:1007930012081D74069000E1F07F017B027A007954
:1007A300E11291387B027A0079E17D057C1A789712
:1007B30012081D74059000E5F0049000E6F07F0236
:0C07C3007B027A0079E112913802068175
:0407CF00E47934F3A2
:1007D3002097067F05129849227934E304F379348C
:0807E300E3B464ECE4FEFF2224
:0A07EB0075D90275E90075F90022C6
:0607F5007F0112906F224B
:10080000A881058118EBC6C908CAC6CA08F67BFFCD
:10081000112ED0E0D0E0D0E0C082C08322D083D0BF
:1008200082EDC0E0ECC0E0E8C0E0C082C083E581BA
:10083000F8241EF58108E8C9CBF709EAF709EBF7B8
:1008400009770009E924F6FA75F000C2D5E924FC1D
:10085000F8E924F9F9ECC0E0E8C0E0D1E512005E67
:10086000FFE92409F9D0E0F8D0E0FCEF605020D592
:1008700074B4250AE4FB74FFFCF7D2D580D3D1FE13
:1008800080CFFF20F71CBCFF067014D2F380C2ECAF
:10089000C0F075F00AA42FD0F030F703F78001FC08
:1008A00080AFB7FF03EF80F4E780E57F00D1FE194A
:1008B0001709800DEF24D0B40A0040C68093B6FF1C
:1008C000EAE581C3941AF581E4FED0E0FFD082D03E
:1008D00083D0E004600ED083D0821581158115810C
:1008E000C082C08322900F78E49360256FA36006D6
:1008F000A350F5A380F293FF400442F080BEE4A32E
:10090000938F83F582E4C2D130F705B7FF027700F9
:100910007340A1D3A380D1EAC8FDE620F703FC8091
:1009200001F71A1AEDF88094D2D17F7880027F58AF
:10093000D17990100421CCBCFF05B7FF02805AC0CA
:10094000F08AF0EAC92419F583E8FEECC0E0D1E5AD
:1009500012005EFF601AC583C9C583F70B19E9C58C
:1009600083F908B800010CEE2404F9E7C39B70E09A
:10097000D0E0FCE5F024FDFAD0F08B82A98309EEEB
:10098000C394FBF583F805828004E7F60809D58255
:10099000F9A9831819C2F0414F8AF0EAC9F583E832
:1009A000FED1E512005EFF6013EEC8CE8D82D1FE4F
:1009B000AD82EEC8CE08B800EA0C80E7A983E5F066
:1009C00024FDFA01487F30D179900806C2F7D18919
:1009D000E8CAC9C88049D2F7EA147D0230F4047D20
:1009E0000424FEF8E68A83A88330E70DD2D1C3E45D
:1009F00096F618DDFAA8838000C2F7D179900A052F
:100A0000D189C9C8CAC9B1FF8015D179E618188043
:100A100004D1797425C2F7F70BCAC9C8CAC2F0E776
:100A2000FDE924002BF8B6300318DBFABB00080BF5
:100A300008BD00031B8013BDFF02800EEDC39BFEAB
:100A40004008600674305192EDFBEB70020148ECF7
:100A5000046023D39B401F601DFE7D2020F13830B1
:100A6000F3027D3030F023BD3018518E18EF30E6A0
:100A700001187111804030F03F71110B30F6390BC5
:100A80008036EF71111E30F6011E518E8028EE6007
:100A900005ED08F6DEFC2230F00771110B30F6018F
:100AA0000BE9FF2419F9E6F71918DBFAEDF719DE5F
:100AB000FCEFF92419F8CCCBEB700201481919E8C6
:100AC000C0E0E6FFD1E50909EFD16AD0E0F818DB14
:100AD000EE090901481A1AD181900F6CE6086002EC
:100AE0002406936023F7190B30E504E4A380F3EBAD
:100AF000C0E0743AF7E924FCF908901004D1891891
:100B0000D0E02405FBE92404C8CAC9E92419F88007
:100B1000AC08EFF68FF030F604743008F622619BD3
:100B2000C2F79159BFFF0261ADEF60F22481FF204F
:100B3000E73618040FD113EBC39F60124010FDFE7F
:100B40000BE89FF8742EC618C6DDFC18805DF4040F
:100B5000FD7E000DE824F9F880057430F6180BDDF1
:100B6000F9742EF60B188043F4FD7E070DBD0700C7
:100B70004016E9FD097430F709E9C39870F7EDF9FB
:100B800080087430F60E0B08DDF8742EF6080B0B97
:100B90007430F6D113E8C39BF88010E92419F87477
:100BA00030F618742EF6187B027E00B1AD414AC2B1
:100BB000F78002D2F79159BFFF0280F1BF000E7497
:100BC00030F618742EF6087E007B02800EEF24812A
:100BD000FF18742EC608C6EBFE1E0BD113E8C39B8C
:100BE000F8EFC0E0B1ADD113D0E0FFC0F0E8C39B97
:0E0BF000F8E730F704746580027445F618EFDC
:100BFE0020E704762B8004762DF4041875F00A8411
:100C0E002430F618E5F02430F6EB2404FBD0F0D1B6
:100C1E002918B1FF61ADC2F78002D2F7D2F2915915
:100C2E00BFFF0261ADE7B4FF037406F7BF7B004060
:100C3E0016EF248120E706C397600C500A74822FAA
:100C4E00C7C397F7020B2917020BBCD179ECC0E092
:100C5E00C0F018E63308E63392D5186033B4FF407F
:100C6E00E6C2E76009900FBCC2D17B078007900FE8
:100C7E00C3D2D17B06E493F709A3DBF97B0330D112
:100C8E000A742B30D502742DF70B09197C80A184C0
:100C9E00EAC0E074307A08F709DAFC097C81A17D9C
:100CAE00CAC0E0EA75F010A4CAABF075F04DA42BE3
:100CBE00FBE435F0FCEA2410FAEB34C5FBEC34D936
:100CCE00FCE6C2E7FF75F056A4F42411C5F0F43427
:100CDE00C58FF0A42AE5F03BE43CFBC0E0E9C0E0A0
:100CEE00E8C0E0EBC0E020E707800812112C801F5F
:100CFE00F404FB121411D0F0D0E0F8C0E0187583A4
:100D0E000418E6C0E008D583F930F7DF121288D058
:100D1E00E0F8D0E02408F9EED2E7CE33EF332482A8
:100D2E00FAECFBD0E0FCE4C3CB33CBCD33CDCE33EA
:100D3E00CE33DAF37A0875F00A8460062430F71998
:100D4E001A0CE5F02430F7198BF0740AA4FBAFF0FF
:100D5E008DF0740AA42FFDAFF050010F8EF0740ABF
:100D6E00A42FFE743035F0F719DADDE9240AF9D034
:100D7E00E0FAE9D39AFBECFF247FFFCAC9C824FD31
:100D8E00FAE9FD09EF046003120F2FEDF909EF04E4
:100D9E006003120F2FEDF9D0F0D0E0FC7B0722E7B5
:100DAE00B4FF027406700820F0010E8E838016C305
:100DBE009E400EF583603674300BF618D583FA809C
:100DCE002CF404F583C0E0E9C0E0E8C0E0F92B04A0
:100DDE00F8EEC0E0EFC0E009120F2DD583FAD0E097
:100DEE00FFD0E0FED0E0F8D0E0F9D0E0FD08D12948
:100DFE0018D2F07F2D20D10C7F2B20F5077F2020DD
:100E0E00F602C2F0228982E92419F98B83E6F719DA
:100E1E0018D583F9A982E92419F822E9F58224016B
:100E2E00F98B8330F22A20F027C2F2E608B42E02A4
:100E3E00D2F2D583F6E8C39BF88B8330F210E6B47A
:100E4E003005081BD583F7B42E07081B8006D2F297
:100E5E00E6F70908D583F9E9F8A98222BDFF051244
:100E6E000240800312002609071922E9CAC8E924A4
:100E7E0001F922E9CAC8E92419F922A2F492D5C0CF
:100E8E00F0E582FD30D50623F582FD181818E685AB
:100E9E0083F084F620D5047B0180027B0308E5F005
:100EAE00D6C6C48583F084C4C6C445F0C48583F019
:100EBE0084D6DBE9E5F024F6500730D10224202455
:100ECE0007243AF70920D509DDC3D0F01818AB82F4
:100EDE0022DDB8181880F3E7F819E7FC19E7FDBD15
:100EEE00FF0122090907B70004190719221919224F
:100EFE00CACDE8C0E0E9C0E0E6FB08E6FA08E6F98C
:100F0E00EFBBFF05120240800A06B6000318060862
:100F1E00120042080618D0E0F9D0E0F8CDCA22E956
:100F2E00FD1BE7B4350FEBFE600709E719F709DE85
:100F3E00F718EDF92240EF09C3E899601AE719B4E2
:100F4E002E04F70980F104B43A067430F70980E7ED
:100F5E00F709E899FE80D1197431F70B80D4286E09
:100F6E00756C6C290049584450434C046C10620057
:100F7E00680023012D022B2020402E80002A091705
:100F8E006F09C578092858092E7309377509F96450
:100F9E0009D66909D6630A0A250A11700AD5660BA5
:100FAE0020650BB3450BAF670C28470C240020209F
:0B0FBE0020204E614E202020464E49AE
:100FC9001200C4EFB2E7FF80031200C4E58124FDDB
:100FD900F8F9E63308E63370060213B60213A504DE
:100FE90060FAEE33EF33700EE6FF18E6FE18E6FD01
:100FF90018E6FC0213B60460E3E58124FBF8D3ECA0
:101009009608ED9608EE9608EFC2E786F0C2F795C6
:10101900F0400FEFC6FF18EEC6FE18EDC6FD18EC3E
:10102900C6FC1213C7C3EB9FF5F0700EE58124FBD4
:10103900F9E4C3CC20D5730211049418605C400E06
:10104900E4FF19E7FE19E7FD19E7FC0210E0E4FFE8
:1010590030F405CEFCE4CDFF30F305E4CECDCCCFA2
:1010690030F21AE5D054184404F8EF54F0D6C4FF0E
:1010790008ECD6C4FC08EDD6C4FDEEC4FE740355D5
:10108900F06012F5F0C3EE13FEED13FDEC13FCEF67
:1010990013FFD5F0F030D55D8009E4CEFFE4FDFC07
:1010A90030D552C3E49FCC191919C797CD09C797F1
:1010B900CE09C797FF4E4D4C70140213B6DB0302DD
:1010C90013A9EC2CFCED33FDEE33FEEF33FFEF30CB
:1010D900E7EBECCFCECDFCEF30E70D0CBC00090DF2
:1010E900BD00050EBE00010BEB7005A2D102139DD8
:1010F900A2D10213B0E42FCC19191937CD0937CE73
:101109000937FF50090BEB700CA2D102139DEFCEEA
:10111900CDCCFF80C2EF13CE13CD13CC13FF80B714
:101129001200C4EF4E601AE58124FEF924FEF8E7A7
:1011390019477019EE33EF33B4FF030213A50213F5
:10114900A9E58124FDF8E63308E63380EB1213C7DD
:10115900248150082B5008A2D502139D2B50DFF78C
:10116900FAE61846197020B7800DEE33CAA2D513D6
:10117900FFCA13FE0213B6EC4D703CBE8046E6FC76
:1011890008E6FD08E680E4EC4D7039BE800280EE89
:10119900E4CEC7CDC6F5F008E4C6CCF9FBFFFA806A
:1011A90076E4CEC9E4CDCAE4FFCCFB803CE4C9CDEA
:1011B900CFCBECCACC8060E4F9FAFBFFCECDCCC52D
:1011C900F00880538CF0E660D8A4C5F0CDFAC5F0DC
:1011D900E6A42DCEF9C5F03400FDE6A42DC5F03402
:1011E90000FDCCFBC5F0CC7F0008E660C0A42EC58D
:1011F900F03C50010DCAFCC5F0CEE6A42AC5F03D6D
:1012090050010FC9FDC5F0CAE6A429C5F03F79010F
:10121900400119CBC5F0CF08E6A42AC5F03F500517
:101229000BBB000109CCC5F0FAE6A42CC5F03B5074
:101239000109CDC5F0CCE6A42DFDC5F039FE330872
:10124900500906B60011A2D502139DEA33FAEC3310
:10125900FCED33FDEE33FEEA30E7140CBC00100D53
:10126900BD000C0EBE000806B60004A2D580D9E662
:05127900A2D50213B034
:10127E00D083D0820213A91200C4EFC2E74E7003CE
:10128E000213A5C082C083E58124FBF8F9E6084667
:10129E0060DE1213C70FBF0006D083D08280E1EF4D
:1012AE0024805007C3CB9B500D80C5CB9B4007D0ED
:1012BE0083D08202139DF6F583EC4D701FBE801C09
:1012CE00E58124FBF8E583A2D513FFE692E7FE182D
:1012DE00E6FD18E6FCD083D0820213B6E58124FB2E
:1012EE00F8E6CEF618E6CDF618E6CCF6EFCCFFE82B
:1012FE002402F9F8E7FA19E7FB19E7FCE4F5F075B3
:10130E00821A758380801DE58303F58330E706A777
:10131E00F009E4F5F0C3EF33FFED33FDEE33FE409D
:10132E000C30E717C3EF9CED9BEE9A400EC3EF9C7B
:10133E00FFED9BFDEE9AFEE58342F0D582C9E7FAFA
:10134E0019E9F81919E720E7191ABA000302127EF3
:10135E00E5F025F0FFE633FC18E633FD18E633FE24
:10136E008009FE09E7FDE6FCE5F0FFEF30E7160C1D
:10137E00BC00120DBD000E0EBE000A0A7007D0830F
:0F138E00D08202139DEAA2D5D083D0820213B081
:10139D0074FF13FF7E80800774FF8001E4FFFEFD64
:1013AD00FC800613FFEE92E7FED0E0F8D0F0E58169
:1013BD0024FCF581C0F0E8C0E022E7D2E7C733098D
:1013CD00E733FB92D592D1EED2E7CE33EF33FF5018
:0413DD0002B2D52261
:1013E1003F8000003DCCCCCD3C23D70A3A83126F1D
:1013F10038D1B7173727C5AC358637BD33D6BF953A
:10140100322BCC7724E69595179ABE150A4FB11F5A
:10141100EB60105407700AEB543803241C12143C7F
:1014210022232312143CEB543870012203241CFBA9
:101431001200ABEB12143C12112C229013E1FC931D
:0E144100FF0CEC93FE0CEC93FD0CEC93FC22E4
:10144F001214958000EC3392D550031214837A2036
:10145F00C3EC20E712EF33FFEE33FEED33FDEC3339
:10146F00FC20E703DAEF22EA247DA2D513FFEC92EA
:10147F00E7CEFC22E4C39FFFE49EFEE49DFDE49CC7
:10148F00FC22C2D580C8EED2E7CE33EF3392D524FB
:10149F0081400CE4C2D5A2D513FC33FDFEFF2224FC
:1014AF00E0500474FF80EFF404FAE4CCCDCECF808B
:1014BF000DC3EF13FFEE13FEED13FDEC13FCDAF18A
:1014CF0020D507EECDFEEFCCFF22E4C39CFCE49DBC
:1014DF00FDE49EFEE49FCCFFEECDFE22EFC2E7FFC0
:1014EF0080A47A083392D5E4FDFEFF30D5031214A1
:1014FF0084EC334010EF33FFEE33FEED33FDEC336E
:10150F00FCDAEE80BEEA247EA2D513CC92E7CDCED4
:03151F00FF80B09A
:10152200E58124FEF88FF063F080E6F96480B5F07F
:101532001B188EF0E6B5F014188DF0E6B5F00D1814
:101542008CF0E6B5F006E4FFFE0213B68FF030F73A
:101552000689F030F701B340077F017E000213B61F
:0715620074FFFFFE0213B647
:101569004241545445525920545950452020202075
:10157900003A4E69434420202020202020202020AA
:1015890020003A4E694D482020202020202020208C
:101599002020003A4C694665202020202020202068
:1015A900202020003A4C69496F202020202020204B
:1015B900202020003A4C69506F2020202020202034
:1015C90020202020003A534C412020202020202098
:1015D900202020202000424154544552592043459F
:1015E9004C4C20202020003A4155544F204445546A
:1015F90045435420202020003A2532642020202011
:1016090020202020202020202000424154542E2038
:1016190043415041434954592020003A2534646DCF
:1016290041682020202020202020004348415247A3
:10163900452043555252454E542020003A253464E2
:101649006D412020202020202020200044495343A0
:10165900482E2043555252454E54202000455849A2
:1016690054204241545445525920202020004E69AB
:1016790043442025326443202534646D4168004E7B
:10168900694D482025326443202534646D41680042
:101699004C694665202025316443202534646D4119
:1016A90068004C69496F2020253164432025346442
:1016B9006D4168004C69506F202025316443202515
:1016C90034646D416800534C412020202531644326
:1016D900202534646D4168005345542042415454D7
:1016E900455259205459504500204E694344202001
:1016F90020202020202020202000204E694D482035
:101709002020202020202020202000204C69466510
:10171900202020202020202020202000204C694942
:101729006F202020202020202020202000204C690C
:10173900506F20202020202020202020200020530E
:101749004C41202020202020202020202020005330
:10175900455420424154544552592043454C4C006C
:101769002025326420202020202020202020202015
:1017790020005345542043415041434954592020A6
:10178900202000202534646D41682020202020205D
:10179900202000202534646D412020202020202095
:1017A9002020004C6F6164204D656D6F7279205B5C
:1017B9002532645D0053617665204D656D6F7279E0
:1017C900205B2532645D004572617365204D656D4E
:1017D9006F72795B2532645D004C6F6164696E6775
:1017E9002062617474657279200066726F6D204D94
:1017F900656D6F7279205B2532645D00204E6F2024
:101809006261747465727920646174610020617425
:10181900204D656D6F7279205B2532645D20004F24
:10182900766572777269746520646174613F20001E
:1018390020536176696E67206261747465727920DC
:101849000020746F204D656D6F7279205B253264BD
:101859005D2000457261736520646174613F2020D9
:101869002020200045726173696E6720626174747B
:1018790065727920002045786974204D454D4F5295
:10188900592020202000204E6943442025326443FA
:10189900202534646D416800204E694D4820253269
:1018A9006443202534646D416800204C69466520F5
:1018B9002025316443202534646D416800204C693A
:1018C900496F202025316443202534646D41680027
:1018D900204C69506F202025316443202534646DE4
:1018E90041680020534C41202020253164432025A4
:1018F90034646D41680020456D707479204D656DC3
:101909006F727920202000202020202020202020F4
:101919002020202020202000457261736520616C01
:101929006C20646174613F200045726173696E6760
:1019390020616C6C20646174610020202066726FE4
:101949006D204D656D6F72792020005345542043F9
:10195900454C4C532044455445435400204155546B
:0D1969004F202020202020202020202000C2
:10197600204D414E55414C20202020202020202063
:10198600005345542043484152474552204D4F4449
:101996004500204359434C45204348415247452082
:1019A60020200020434841524745204F4E4C5920A5
:1019B6002020200020444953434841524745204FA8
:1019C6004E4C592000534554204348415247452028
:1019D6004359434C450053455420534F554E4420DC
:1019E600564F4C554D4500204F4E2020202020209C
:1019F6002020202020202000204F46462020202086
:101A060020202020202020200053455420545249D5
:101A160047474C45204D4F44450020202A2A204563
:101A260052524F52202A2A2020200020204D656D38
:101A36006F7279204661696C20202000204C4F414E
:101A46004420202020205341564520200020534189
:101A56005645202020202045524153452000204550
:101A66005241534520202020464F524D41540020DC
:101A7600464F524D415420202045584954202000BD
:101A8600204558495420202020204C4F41442020F6
:101A960000557365203C3E20746F2053656C65636A
:101AA6007400204E6F74204170706C696361626CC3
:101AB600652000466F722054686973204261747411
:101AC6006572790020466F722054686973204D6FE5
:101AD60064652020002043454C4C53204445544522
:101AE6004354494F4E003A4155544F202020202060
:101AF600202020202020003A4D414E55414C2020E8
:101B060020202020202020002043484152474552D3
:101B1600204D4F4445202020003A4359434C452050
:101B2600434841524745202020003A434841524706
:101B360045204F4E4C5920202020003A444953431B
:101B46004841524745204F4E4C59200020434841BA
:101B5600524745204359434C45202020003A4E6FBA
:101B660074204170706C696361626C65200020535B
:101B76004F554E4420564F4C554D45202020003A97
:101B86004F4E202020202020202020202020200012
:101B96003A4F4646202020202020202020202020AA
:101BA600002054524947474C45204D4F444520207C
:101BB60020002045584954204F5054494F4E532039
:101BC600202000204241545445525920204D454D75
:101BD6004F525900204D454D4F525920204F5054D9
:101BE600494F4E5300204F5054494F4E532020200A
:101BF6002045584954002045584954202020204269
:101C0600415454455259002020534D4152542043CB
:101C160048415247455220002020534552564943D9
:101C260045204D4F44452020002020202046495283
:101C36004D57415245202020200020205645525322
:101C4600494F4E20312E313820200020444953433D
:101C56004820432D53544550202020003A25346413
:101C66002020202020202020202020002043555204
:101C760052454E54205354455020202000205354A2
:101C86004152542044454C415920202020003A25F9
:101C96003364205365636F6E647320202020002018
:101CA60044495343482D4348472044454C41590035
:101CB600204D41582E20564F4C542F43454C4C2016
:101CC600003A25352E32665620202020202020205E
:101CD6002020003A44495341424C452020202020F0
:101CE60020202000204D494E2E20564F4C542F4385
:101CF600454C4C2000204E6943442053454E5349E1
:101D06005449564520003A253264206D562F4365C6
:101D16006C6C20202020202000205043204C494E6F
:101D26004B2020202020202020003A454E41424CC6
:101D360045202020202020202020002053555050D0
:101D46004C59204D4F4E49544F5220003A43482596
:101D560031642020202025352E326656732000203F
:101D6600564F4C544147452053544550202020009F
:101D76003A2534642020202025352E326656200050
:101D8600205741544348444F472054494D4552201B
:101D96000020455849542053455256494345202072
:101DA600200053455420444953434820432D53545F
:101DB6004550005345542043555252454E542053E6
:101DC60054455000534554205354415254204445E1
:101DD6004C415920005345542044495343482D4310
:101DE600484152474500534554204D41582E2056F0
:101DF6002F43454C4C20003A25352E32665620207E
:101E06002020202020202000534554204D494E2ECE
:101E160020562F43454C4C20004E694344205345E1
:101E26004E5349544956452020003A253264206DC8
:101E360056202020202020202020200053455420FA
:101E46005043204C494E4B20202020200020454E58
:101E560041424C45202020202020202020002044E4
:101E6600495341424C452020202020202020005369
:101E7600455420535550504C59204D4F4E2E20005E
:101E860053455420564F4C544147452053544550D2
:101E960000534554205741544348444F472020207F
:021EA60020001A
:071EA8007803EFF21207F5C9
:101EAF009000DEE0B403028074500CE06017146001
:101EBF001414603F021F7EE024FC60611470030263
:051ECF001F55021F7EFB
:101ED4009000DF7405F0A37478F07401900116F09B
:101EE400740C7904F37905740FF30974A0F379077A
:101EF4007407F30974D0F374017909F3807C9000BA
:101F0400DF740EF0A37410F07402900116F07404E0
:101F14007904F37905740FF30974A0F37907E4F3F2
:101F240009F3047909F380529000DF7410F0A3746C
:101F340068F07402900116F0047904F37905740FC3
:101F4400F30974A0F37907E4F309F3047909F3803E
:101F5400299000DF7409F0A37492F07402900116C2
:101F6400F074067904F37905741BF3097458F37952
:101F740007E4F309F374037909F3129201EF790A80
:101F8400F3E3B40403E3FF227903E314601B147046
:101F9400030223E51470030224621470030226CBA7
:091FA4001470030227CE021EAFE7
:101FAD007F017B057A1679E1129138790AE3B40144
:011FBD00150E
:101FBE009000DEE0B40001D34005E014F08006741A
:101FCE00059000DEF0790AE3B402028003022330AA
:101FDE009000DEE0FAB4030302206F500CEA6017A3
:101FEE001460311460650220DBEA24FC6073147007
:071FFE00030220A50220DB15
:102005009000D37403F0A374E8F09000D3E0FAA332
:10201500E0FB9000DAEAF0A3EBF00220DB9000D3BE
:102025007407F0A304F0E4FCFD9000D3E0FEA3E008
:10203500FF121491C004C005C006C007E4FEFCFDF4
:10204500743FFF12112C121495EE9000DAF0A3EFF5
:10205500F00220DB9000D37408F0A374FCF090002C
:10206500DA740BF0A374B8F0806C9000D37408F0A8
:10207500A374FCF0E4FCFD9000D3E0FEA3E0FF12A6
:102085001491C004C005C006C0077433FEFCFD747E
:102095003FFF12112C121495EE9000DAF0A3EFF029
:1020A5009000D37405F0A37414F0E4FCFD9000D304
:1020B500E0FEA3E0FF121491C004C005C006C007EE
:1020C500E4FCFD7440FE14FF12112C121495EE90E1
:1020D50000DAF0A3EFF09000DAE0FAA3E0BA00032B
:1020E500B4640050099000DAE4F0A37464F0900041
:1020F500DAE0FEA3E0FFE4FC7D64120179EE9000D6
:10210500DAF0A3EFF09000DAE0FEA3E0FFE4FC7D57
:102115006412013DEE9000DAF0A3EFF0BE0B04BFB0
:10212500B801D3400A9000DA740BF0A374B8F090AC
:1021350000D3E0F5F0A3E0FB7905E3B5F00509E38D
:10214500B50300500B79059000D3E3F009A3E3F044
:102155007F05129849EE790BF309EFF3E4FCFD9046
:10216500011EE0FEA3E0FF121491C004C005C006E5
:10217500C00774CDFC14FDFE743DFF12112C790DC2
:102185001200F4E4FCFD790BE3FE09E3FF12149160
:10219500C004C005C006C007780D1200DC12128805
:1021A500C004C005C006C0077466FEFCFD743FFF91
:0B21B500121522BF0102800302232349
:1021C0009000DEE0B40303022287500CE0601A1492
:1021D0006017146063022321E024FC70030222874D
:0921E0001470030222D502232A27
:1021E900E4FCFD790BE3FE09E3FF121491C004C07E
:1021F90005C006C007780D1200DC121288C004C0A1
:1022090005C006C0077CF57DBE7E207F4012112CDB
:10221900C004C005C006C00774ABFC14FDFE743EC3
:10222900FF12112C121495EF9000D5F002232AE425
:10223900FCFD790BE3FE09E3FF121491C004C0050C
:10224900C006C007780D1200DC121288C004C00550
:10225900C006C0077CB07DDE7E687F3F12112CC0AE
:1022690004C005C006C00774ABFC14FDFE743EFF34
:1022790012112C121495EF9000D5F002232AE4FCD8
:10228900FD790BE3FE09E3FF121491C004C005C0F8
:1022990006C007780D1200DC121288C004C005C000
:1022A90006C0077C4D7D187E807F3F12112CC0042B
:1022B900C005C006C00774ABFC14FDFE743EFF12D6
:1022C900112C121495EF9000D5F08055E4FCFD799E
:1022D9000BE3FE09E3FF121491C004C005C006C058
:1022E90007780D1200DC121288C004C005C006C0B0
:1022F900077C207D527EC07F3F12112CC004C0058F
:10230900C006C00774ABFC14FDFE743EFF12112C0D
:0A231900121495EF9000D5F0800734
:102323007909E39000D5F01291EEE4FF22790AE3F4
:03233300B40313DD
:102336009000DEE0B405005005E004F08005E4906E
:1023460000DEF09000DEE0700F7B027A0079E17D1E
:10235600057C1678F212081D9000DEE0FAB4010F33
:102366007B027A0079E17D057C17780312081D90BF
:1023760000DEE0FAB4020F7B027A0079E17D057C8B
:1023860017781412081D9000DEE0FAB4030F7B02E2
:102396007A0079E17D057C17782512081D9000DE0C
:1023A600E0FAB4040F7B027A0079E17D057C1778A8
:1023B6003612081D9000DEE0FAB4050F7B027A00A3
:1023C60079E17D057C17784712081D74069000E1B7
:1023D600F07F027B027A0079E1129138021EAF7F0C
:1023E600017B057A177958129138790AE3B40115F9
:1023F6007909E3F5F09000D5E0B5F001D3400690F9
:0B24060000D5E014F0790AE3B40206F0
:102411001291EEE4FF22790AE3B403147904E3F59F
:10242100F09000D5E0B5F00050069000D5E004F042
:102431009000D5E0FBE4C0E0C0037B027A0079E1C3
:102441007D057C17786912081D1581158174069028
:1024510000E1F07F027B027A0079E1129138021EDD
:10246100AF7F017B057A17797B1291389000D3E019
:10247100FAA3E0BA0003B4640050099000D3E4F079
:10248100A37464F09000D3E0F5F0A3E0FB7905E3D9
:10249100B5F00509E3B50300500B79059000D3E3CE
:1024A100F009A3E3F0790AE3B401209000D3E0B48A
:1024B1000006A3E0B46401D340119000D4E024CE1F
:1024C100FB9000D3E034FFF0A3EBF0790AE3B40210
:0624D10002800302266CEC
:1024D7009000DEE070109000D3E0FAA3E0FB9000DC
:1024E700DAEAF0A3EBF09000DEE0FAB4011F900007
:1024F700D3E0B40306A3E0B4E801D350109000D3AF
:10250700E0FAA3E0FB9000DAEAF0A3EBF09000DE3C
:10251700E0FAB4013E9000D3E0B40306A3E0B4E8C8
:1025270001D3402F9000D3E0FAA3E0FBE4FCFDAE1B
:1025370002AF03121491C004C005C006C007E4FE31
:10254700FCFD743FFF12112C121495EE9000DAF087
:10255700A3EFF09000DEE0B4022C9000D3E0FEA3DE
:10256700E0FFE4FCFD121491C004C005C006C007DB
:102577007C147DAE7EA77F3F12112C121495EE902E
:1025870000DAF0A3EFF09000DEE0FA64036003BA2C
:10259700042C9000D3E0FEA3E0FFE4FCFD121491AD
:1025A700C004C005C006C0077433FEFCFD743FFFBE
:1025B70012112C121495EE9000DAF0A3EFF09000B0
:1025C700DEE0B4052C9000D3E0FEA3E0FFE4FCFDC1
:1025D700121491C004C005C006C007E4FCFD744096
:1025E700FE14FF12112C121495EE9000DAF0A3EFEF
:1025F700F09000DAE0FAA3E0BA0003B464005009EF
:102607009000DAE4F0A37464F0E4FCFD9000DAE0F3
:10261700FEA3E0FF121491C004C005C006C0077CEA
:102627000A7DD77E237F3C12112C121495EE900061
:10263700DAF0A3EFF09000DAE0FEA3E0FFE4FC7D20
:102647006412013DEE9000DAF0A3EFF0BE0B04BF79
:10265700B801D3400A9000DA740BF0A374B8F012F3
:1026670091EEE4FF22790AE3B403289000D37905B9
:10267700E3F5F0E0B5F00909E3F5F0A3E0B5F00004
:1026870050119000D4E02432FB9000D3E03400F0E6
:10269700A3EBF09000D3E0C0E0A3E0C0E07B027AB8
:1026A7000079E17D057C17788C12081D158115814D
:1026B70074069000E1F07F027B027A0079E11291C3
:1026C70038021EAF7F017B057A1679341291389054
:1026D70000DAE0FAA3E0BA0003B4640050099000FE
:1026E700DAE4F0A37464F09000DAE0FAA3E0BA0B3E
:1026F70004B4B801D3400A9000DA740BF0A374B89D
:10270700F0790AE3B4015E9000DAE0B40006A3E0D2
:10271700B46401D3404FE4FCFD9000DAE0FEA3E08F
:10272700FF121491C004C005C006C0079000D3E48F
:10273700FCFDE0FEA3E0FF121491C004C005C00633
:10274700C00774CDFC14FDFE743DFF12112C121549
:1027570022BF01119000DBE0249CFB9000DAE034FB
:0B276700FFF0A3EBF0790AE3B40206D8
:102772001291EEE4FF22790AE3B4031F9000DAE03B
:10278200B40B05A3E0B4B80050119000DBE0246460
:10279200FB9000DAE03400F0A3EBF09000DAE0C046
:1027A200E0A3E0C0E07B027A0079E17D057C177846
:1027B2009C12081D1581158174069000E1F07F02BC
:1027C2007B027A0079E1129138021EAF7F017B050C
:1027D2007A1679551291389000DCE0FAA3E0BA003B
:1027E20003B4640050099000DCE4F0A37464F0794F
:1027F2000AE3B401209000DCE0B40006A3E0B46474
:1028020001D340119000DDE0249CFB9000DCE03419
:0B281200FFF0A3EBF0790AE3B402062C
:10281D001291EEE4FF22790AE3B403287907E3F578
:10282D00F09000DCE0B5F00909E3F5F0A3E0B5F0B8
:10283D000050119000DDE02464FB9000DCE03400DA
:10284D00F0A3EBF09000DCE0C0E0A3E0C0E07B0281
:10285D007A0079E17D057C17789C12081D1581158C
:10286D008174069000E1F07F027B027A0079E1121B
:05287D009138021EAFBE
:102882007811EFF27912E4F30904F37914E4F3090D
:102892007410F319E3FE09E3FF129607EE7916F3BB
:1028A20009EFF37915E32401FF19E33400FE1296D0
:1028B20007EF9000AFF07915E32402FF19E334002B
:1028C200FE129607EE9000A4F0A3EFF07915E32430
:1028D20003FF19E33400FE129607EF9000A6F012F0
:0228E20007F5F8
:1028E400129201EF7918F37911E314600E14600B5E
:0B28F40014600814700302329D80E5A0
:1028FF007911E3B4011C7912E3C0E009E3C0E07B76
:10290F00027A0079E17D057C1778AC12081D1581DC
:10291F0015817911E3B4021C7912E3C0E009E3C019
:10292F00E07B027A0079E17D057C1778BE12081DE5
:10293F00158115817911E3B4031C7912E3C0E00905
:10294F00E3C0E07B027A0079E17D057C1778D01235
:10295F00081D158115817918E3B401028003022A3D
:10296F000F7912E3B4000609E3B40001D350030258
:02297F002A0F1D
:102981007913E314F3F4197003E314F37912E3B444
:0A299100000609E3B40001D3406C16
:10299B007913E324FFFF19E334FFFEE4FC7D0A12F5
:1029AB00013DEF2410FFE43E7914F309EFF319E333
:1029BB00FE09E3FF129607EE7916F309EFF379158B
:1029CB00E32401FF19E33400FE129607EF9000AFEA
:1029DB00F07915E32402FF19E33400FE129607EE9B
:1029EB009000A4F0A3EFF07915E32403FF19E3346F
:0C29FB0000FE129607EF9000A6F0800886
:102A07007912E4F309740BF37918E3B40202800333
:032A17000230206A
:102A1A007912E3B4000809E3B40B03E4FF22791145
:092A2A00E3B401028003022B8CCD
:102A33007813E22400FB18E23455F5F07916E3B578
:102A4300F0028003022B4309E3B503028003022B48
:012A5300433F
:102A54007F017B057A1779E21291387912E3C0E09D
:102A640009E3C0E07B027A0079E17D057C1778F305
:102A740012081D158115817F027B027A0079E1120B
:102A840091387913E324FFFF19E334FFFEE4FC7D5E
:102A94000A12013DEF2410FFE43E7914F309EFF329
:102AA400E32401FF19E33400FE129607EF9000DEE1
:102AB400F07915E32402FF19E33400FE129607EEC1
:102AC4009000D3F0A3EFF07915E32403FF19E33466
:102AD40000FE129607EF9000D5F07915E32404FF69
:102AE40019E33400FE129607EE9000DAF0A3EFF03B
:102AF4007915E32405FF19E33400FE129607EE90DE
:102B040000DCF0A3EFF07915E32406FF19E33400A9
:102B1400FE129607EE9000DFF0A3EFF0129698E411
:102B2400FE7F0E1296F1E4FE7F0E7912E3FC09E3B8
:0F2B3400FD1295CE1297191291EED208E4FF22EE
:102B43001291EE7F017B057A18790512913879127B
:102B5300E3C0E009E3C0E07B027A0079E17D057C14
:102B630018781612081D158115817F027B027A00E1
:102B730079E1129138E4FE7F641291D61291EE7ED0
:102B8300057FDC1291D6E4FF227911E3B4020280BF
:042B930003022E35D6
:102B97007813E22400FB18E23455F5F07916E3B513
:102BA700F0028003022D2E09E3B503028003022DF4
:012BB7002EEF
:102BB8007B057A187928128E97EF64016003022E3C
:012BC80035D7
:102BC9007F017B057A1879391291387912E3C0E0CF
:102BD90009E3C0E07B027A0079E17D057C18784A37
:102BE90012081D158115817F027B027A0079E11295
:102BF90091381296987913E324FFFF19E334FFFE05
:102C0900E4FC7D0A12013DEF2410FFE43E7914F340
:102C190009EFF319E3FE09E3FF1296F17915E324AD
:102C290001FF19E33400FE1296F17915E32402FF3E
:102C390019E33400FE1296F17915E32403FF19E331
:102C49003400FE1296F17915E32404FF19E33400E8
:102C5900FE1296F17915E32405FF19E33400FE12FB
:102C690096F17915E32406FF19E33400FE1296F173
:102C79007914E3FE09E3FF7813E22400FD18E23436
:102C890055FC1295CE7915E32401FF19E33400FEB2
:102C99009000DEE0FD7C001295CE7915E32402FF59
:102CA90019E33400FE9000D3E0FCA3E0FD1295CEB9
:102CB9007915E32403FF19E33400FE9000D5E0FD04
:102CC9007C001295CE7915E32404FF19E33400FE44
:102CD9009000DAE0FCA3E0FD1295CE7915E3240516
:102CE900FF19E33400FE9000DCE0FCA3E0FD12953F
:102CF900CE7915E32406FF19E33400FE9000DFE0E6
:102D0900FCA3E0FD1295CEE4FE7F0E1296F1E4FEDF
:102D19007F0E7912E3FC09E3FD1295CE1297191281
:052D290091EEE4FF2221
:102D2E007F017B057A1879391291387912E3C0E068
:102D3E0009E3C0E07B027A0079E17D057C18784AD0
:102D4E0012081D158115817F027B027A0079E1122E
:102D5E0091381296987913E324FFFF19E334FFFE9E
:102D6E00E4FC7D0A12013DEF2410FFE43E7914F3DA
:102D7E0009EFF319E3FE09E3FF7913E32400FD19CC
:102D8E00E33455FC1295CE7915E32401FF19E33493
:102D9E0000FE9000DEE0FD7C001295CE7915E32456
:102DAE0002FF19E33400FE9000D3E0FCA3E0FD1215
:102DBE0095CE7915E32403FF19E33400FE9000D578
:102DCE00E0FD7C001295CE7915E32404FF19E3345F
:102DDE0000FE9000DAE0FCA3E0FD1295CE7915E33B
:102DEE002405FF19E33400FE9000DCE0FCA3E0FDB7
:102DFE001295CE7915E32406FF19E33400FE9000F8
:102E0E00DFE0FCA3E0FD1295CEE4FE7F0E1296F1FC
:102E1E00E4FE7F0E7912E3FC09E3FD1295CE1297C4
:102E2E00191291EEE4FF227911E3B403028003023A
:022E3E00302042
:102E40007813E22400FB18E23455F5F07916E3B567
:102E5000F0028003022F4909E3B503028003022F29
:012E60004928
:102E61007B057A18795C128E97EF6401600302305A
:012E71002040
:102E72007F017B057A18796D1291387912E3C0E0EF
:102E820009E3C0E07B027A0079E17D057C1778F3E3
:102E920012081D158115817F027B027A0079E112E9
:102EA20091381296987913E324FFFF19E334FFFE59
:102EB200E4FC7D0A12013DEF2410FFE43E7914F395
:102EC20009EFF319E3FE09E3FF1296F17915E32402
:102ED20001FF19E33400FE1296F17915E32402FF93
:102EE20019E33400FE1296F17915E32403FF19E386
:102EF2003400FE1296F17915E32404FF19E334003D
:102F0200FE1296F17915E32405FF19E33400FE124F
:102F120096F17915E32406FF19E33400FE1296F1C7
:102F22007915E32407FF19E33400FE1296F1E4FE5B
:102F32007F0E1296F1E4FDFEFC7F0E1295CE1297E3
:072F4200191291EEE4FF22D9
:102F49007F017B057A18796D1291387912E3C0E017
:102F590009E3C0E07B027A0079E17D057C1778F30B
:102F690012081D158115817F027B027A0079E11211
:102F790091381296987913E324FFFF19E334FFFE81
:102F8900E4FC7D0A12013DEF2410FFE43E7914F3BD
:102F990009EFF319E3FE09E3FF1296F17915E3242A
:102FA90001FF19E33400FE1296F17915E32402FFBB
:102FB90019E33400FE1296F17915E32403FF19E3AE
:102FC9003400FE1296F17915E32404FF19E3340065
:102FD900FE1296F17915E32405FF19E33400FE1278
:102FE90096F17915E32406FF19E33400FE1296F1F0
:102FF9007915E32407FF19E33400FE1296F1E4FE84
:103009007F0E1296F1E4FDFEFC7F0E1295CE12970B
:10301900191291EEE4FF227918E3B4030280030246
:1030290030CF7912E3B4000509E3B40C0040030280
:0230390030CF96
:10303B007913E304F3197003E304F37912E3B40097
:10304B000C09E3B40C077912E4F30904F37912E3E6
:0A305B00B4000509E3B40B00506A4D
:103065007913E324FFFF19E334FFFEE4FC7D0A1224
:10307500013DEF2410FFE43E7914F309EFF319E362
:10308500FE09E3FF129607EE7916F309EFF37915BA
:10309500E32401FF19E33400FE129607EF9000AF19
:1030A500F07915E32402FF19E33400FE129607EECA
:1030B5009000A4F0A3EFF07915E32403FF19E3349E
:1030C50000FE129607EF9000A6F07912E3B4001AFD
:0530D50009E3B40B1536
:1030DA007B027A0079E17D057C18787E12081D74DE
:1030EA00069000E1F07F017B027A0079E1129138C3
:1030FA007918E3B404037F04227813E22400FB184E
:10310A00E23455F5F07916E3B5F002800302325F36
:0A311A0009E3B50302800302325FEF
:103124009000AFE0B403030231CB500CE0601A14FA
:103134006041146068023244E024FC70030231F4FC
:0931440014700302321D02324432
:10314D009000A4E0C0E0A3E0C0E0A3E0FBE4C0E099
:10315D00C0037B027A0079E17D057C18788F120817
:10316D001D74FC2581F5810232449000A4E0C0E07D
:10317D00A3E0C0E0A3E0FBE4C0E0C0037B027A0063
:10318D0079E17D057C1878A112081D74FC2581F567
:10319D00810232449000A4E0C0E0A3E0C0E0A3E0CF
:1031AD00FBE4C0E0C0037B027A0079E17D057C1869
:1031BD0078B312081D74FC2581F58102324490000C
:1031CD00A4E0C0E0A3E0C0E0A3E0FBE4C0E0C003E6
:1031DD007B027A0079E17D057C1878C612081D7492
:1031ED00FC2581F58180509000A4E0C0E0A3E0C0F3
:1031FD00E0A3E0FBE4C0E0C0037B027A0079E17D4F
:10320D00057C1878D912081D74FC2581F58180275D
:10321D009000A4E0C0E0A3E0C0E0A3E0FBE4C0E0C8
:10322D00C0037B027A0079E17D057C1878EC1208E9
:10323D001D74FC2581F5819000D5E0600790010C8F
:04324D00E0B4011DCB
:0E32510074209000E7F074419000E8F0800FC8
:10325F007B027A0079E17D057C1878FF12081D74D6
:10326F00069000E1F07912E3B4000509E3B40B0016
:10327F00500E7F027B027A0079E11291380233D926
:10328F007F027B057A1979101291380228E47B05A9
:0F329F007A197921128E97EF640160030233D9F7
:1032AE007F017B057A1979321291387F027B057A7C
:1032BE001979431291381296981296AEE4FE7F64F5
:1032CE001291D6E4FDFEFF7C011295CEE4FE7F0145
:1032DE0090010CE0FD7C001295CE900116E0FBE40F
:1032EE007914F309EBF3900119E0B4010C7915E3AD
:1032FE004480FB19E3F309EBF390011BE0B4010CDE
:10330E007915E34440FB19E3F309EBF3E4FE7F0286
:10331E007914E3FC09E3FD1295CEE4FE7F039001E0
:10332E001CE0FD7C001295CEE4FE7F0490011DE0B2
:10333E00FD7C001295CEE4FE7F05900113E0FCA308
:10334E00E0FD1295CEE4FE7F06900109E0FCA3E0BD
:10335E00FD1295CEE4FE7F0790011EE0FCA3E0FD7A
:10336E001295CEE4FE7F08900110E0FCA3E0FD1262
:10337E0095CEE4FE7F09900117E0FD7C001295CEFC
:10338E00E4FE7F0A900120E0FD7C001295CEE4FE63
:10339E007F0B90011AE0FD7C001295CEE4FE7F0CAF
:1033AE0090010DE0FD7C001295CEE4FE7F0D9001A4
:1033BE000EE0FCA3E0FD1295CEE4FDFEFC7F0E12A6
:0E33CE0095CE1297191291EEE4FF220228E428
:0733DC007819EFF21207F56A
:1033E300129201EF791AF3E3B404037F04227919EB
:1033F300E314601A1470030234A3147003023567D4
:0E3403001470030235E214700302367480D296
:103411007F017B057A19795412913890010CE0B43F
:1034210001117B027A0079E17D057C19786512082A
:103431001D800F7B027A0079E17D057C1978761277
:10344100081D74069000E1F07F027B027A0079E1A9
:0E345100129138791AE364016004E3B40311A8
:10345F0090010CE0B40104E4F08006740190010CBB
:0C346F00F0791AE3B40202800302372552
:07347B00900115E0B4011BF4
:10348200129698E4FE7F011296F1E4FE7F0190010C
:103492000CE0FD7C001295CE1297191291EEE4FF1A
:1034A200227F017B057A197987129138791AE3B460
:0234B200011502
:1034B400900116E0B40101D34005E014F0800674D5
:0B34C40003900116F0791AE3B402280F
:0734CF00900115E0B4011BA0
:1034D600129698E4FE7F021296F1E4FE7F029001B6
:1034E60016E0FD7C001295CE1297191291EEE4FFBC
:0734F60022791AE3B403146C
:1034FD00900116E0B403005005E004F0800674015D
:10350D00900116F0900116E0B4010F7B027A00795C
:10351D00E17D057C19789812081D900116E0B40222
:10352D000F7B027A0079E17D057C1978A912081DBF
:10353D00900116E0B4030F7B027A0079E17D057CE2
:10354D001978BA12081D74069000E1F07F027B0213
:10355D007A0079E11291380233E37F017B057A1904
:10356D0079CB12913890010BE0FBE4C0E0C0037BF6
:10357D00027A0079E17D057C16780112081D15810E
:10358D00158174069000E1F07F027B027A0079E1EB
:10359D00129138791AE3B4011090010BE0B40101D6
:0F35AD00D3400690010BE014F0791AE3B4020644
:1035BC001291EEE4FF22791AE3B40302800302377E
:1035CC002590010BE0B40A00400302372590010B53
:1035DC00E004F00233E37F017B057A1979DC129168
:1035EC003890011CE0B401117B027A0079E17D0571
:1035FC007C1978ED12081D800F7B027A0079E17D31
:10360C00057C1978FE12081D74069000E1F07F020B
:10361C007B027A0079E1129138791AE36401600433
:04362C00E3B40311EF
:1036300090011CE0B40104E4F08006740190011CC8
:0C364000F0791AE3B4020280030237257F
:07364C00900115E0B4011B21
:10365300129698E4FE7F031296F1E4FE7F03900135
:103663001CE0FD7C001295CE1297191291EEE4FF37
:10367300227F017B057A1A790F12913890011BE0A2
:10368300B401117B027A0079E17D057C1978ED1292
:10369300081D800F7B027A0079E17D057C1978FE95
:1036A30012081D74069000E1F07F027B027A007914
:0F36B300E1129138791AE364016004E3B4031162
:1036C20090011BE0B40104E4F08006740190011B38
:0736D200F0791AE3B4024C89
:0736D900900115E0B4013F70
:1036E000900116E0791BF3900119E0B40108791BF1
:1036F000E34480791BF390011BE0B40108791BE3DC
:103700004440791BF3129698E4FE7F021296F1E48E
:10371000FE7F02791BE3FD7C001295CE12971912F1
:0837200091EEE4FF220233E305
:083728007401791FF31207F58B
:10373000129201EF7920F3E31460121460281470E0
:0D374000030237EF14700302380502380849
:10374D00791FE3B40101D34008791FE314F3023864
:0F375D00087406791FF3023808791FE3B40606D3
:06376C001207F5E4FF2244
:10377200791FE364026009E364036004E3B405298A
:0A3782009000DEE0B40101D3401F07
:10378C007F017B057A1A79A81291387F027B057A22
:10379C001A79B91291387E077FD01291D6803F7971
:0D37AC001FE3B40327900116E06401601FC5
:1037B9007F017B057A1A79A81291387F027B057AF5
:0F37C9001A79CA1291387E077FD01291D68012DA
:1037D800791FE3FF1233DCEF7821F2E2B404037FB0
:1037E80004221207F58019791FE3B40600500779FF
:1037F8001FE304F3800A7401791FF380037F042216
:10380800791FE3B404030239435010E314601D1414
:10381800605D1470030238D50239FDE324FB7003A0
:0C3828000239861470030239D2023730D6
:103834007B027A0079E17D057C1A78DB12081D741D
:10384400069000E1F07F017B027A0079E112913861
:1038540090010CE0B4010E7F027B057A1A79EC1218
:1038640091380239FD7F027B057A1A79FD1291386D
:103874000237307B027A0079E17D057C1B780E12D9
:10388400081D74069000E1F07F017B027A0079E163
:10389400129138900116E0B4010B7F027B057A1B6C
:1038A400791F129138900116E0B4020B7F027B0558
:1038B4007A1B7930129138900116E0B40302800328
:1038C4000239FD7F027B057A1B7941129138023758
:1038D400307B027A0079E17D057C1B785212081D49
:1038E40074069000E1F07F017B027A0079E1129185
:1038F400389000DEE0B40101D35008900116E06472
:103904000160117B027A0079E17D057C1B786312EA
:10391400081D801D90010BE0FBE4C0E0C0037B02A6
:103924007A0079E17D057C16780112081D15811550
:10393400817F027B027A0079E11291380237307B71
:10394400027A0079E17D057C1B787412081D7406E7
:103954009000E1F07F017B027A0079E112913890C6
:10396400011CE0B4010E7F027B057A1B798512915C
:10397400380239FD7F027B057A1B79961291380251
:1039840037307B027A0079E17D057C1B78A7120829
:103994001D74069000E1F07F017B027A0079E11248
:1039A400913890011BE0B401179000DEE0B40101EE
:1039B400D3500D7F027B057A1B79851291388039AB
:1039C4007F027B057A1B79961291380237307B028D
:1039D4007A0079E17D057C1B78B812081D74069085
:1039E40000E1F07F017B027A0079E11291387F02D5
:0C39F4007B057A197910129138023730E7
:073A0000E47922F31207F53F
:103A0700129201EF7923F3E314600C14602214700F
:073A170003023AB8023ACBAA
:103A1E007922E3B40001D340087922E314F3023A89
:103A2E00CB74037922F3023ACB7922E3600C146053
:0A3A3E002B14604E14606D023ACBA9
:103A4800120271EF7924F31207F57924E3B4045EC6
:103A58001291EE308003208155E4FE7F641291D6E6
:103A680080F1120679EF7924F31207F57924E3B48B
:023A7800041236
:103A7A001291EE308003208109E4FE7F641291D610
:103A8A0080F130082722123728EF7924F31207F53C
:063A9A007924E3B40416D8
:103AA0001291EE30800320810DE4FE7F641291D6E6
:103AB00080F11207F52280137922E3B40300500746
:103AC0007922E304F38004E47922F37922E3600BA2
:0B3AD000146019146027146035804258
:103ADB007B027A0079E17D057C1B78C912081D8079
:103AEB00317B027A0079E17D057C1B78DA12081DA7
:103AFB0080207B027A0079E17D057C1B78EB120834
:103B0B001D800F7B027A0079E17D057C1B78FC120E
:103B1B00081D74069000E1F07F017B027A0079E1C9
:103B2B001291387B027A0079E17D057C1A78971225
:103B3B00081D74059000E5F0049000E6F07F027B11
:0B3B4B00027A0079E1129138023A077B
:103B56007F017B057A1C790D1291387F027B057AED
:103B66001C791E1291387E057FDC1291D67F017B6F
:103B7600057A1C792F1291387F027B057A1C7940D1
:103B86001291387E057FDC1291D6E47925F312076F
:013B9600F539
:103B9700129201EF7926F3E314600814601C146095
:033BA7002F80402C
:103BAA007925E3B40001D340077925E314F3803083
:0D3BBA00740B7925F380297925E3B40B0401
:043BC7001207F522CA
:103BCB007925E3FF1240741207F580137925E3B4CE
:103BDB000B0050077925E304F38004E47925F3798E
:103BEB0025E3B40C004003024071FA232A903BFCFE
:103BFB0073023C23023C6E023CB9023D04023D4F72
:103C0B00023DD9023E45023E90023ED3023F6D0279
:083C1B004004024046023B9701
:103C23007B027A0079E17D057C1C785112081D74B2
:103C3300069000E1F07F017B027A0079E11291386E
:103C430090010EE0C0E0A3E0C0E07B027A0079E1DE
:103C53007D057C1C786212081D158115817F027B0E
:103C6300027A0079E1129138023B977B027A00795C
:103C7300E17D057C1C787212081D74069000E1F04A
:103C83007F017B027A0079E1129138900109E0C04B
:103C9300E0A3E0C0E07B027A0079E17D057C1C783B
:103CA3006212081D158115817F027B027A0079E17A
:103CB300129138023B977B027A0079E17D057C1CE7
:103CC300788312081D74069000E1F07F017B027A6D
:103CD3000079E112913890011AE0FBE4C0E0C003DF
:103CE3007B027A0079E17D057C1C789412081D150E
:103CF3008115817F027B027A0079E1129138023BC0
:103D0300977B027A0079E17D057C1C78A512081D5A
:103D130074069000E1F07F017B027A0079E1129151
:103D23003890010DE0FBE4C0E0C0037B027A007928
:103D3300E17D057C1C789412081D158115817F0295
:103D43007B027A0079E1129138023B977B027A0079
:103D530079E17D057C1C78B612081D74069000E19C
:103D6300F07F017B027A0079E1129138900113E030
:103D7300FAA3E0FBBA0704B46C01D3503CE4FCFDA6
:103D8300AE02AF03121491C004C005C006C0077C85
:103D93006F7D127E837F3A12112CC004C005C006CA
:103DA300C0077B027A0079E17D057C1C78C7120885
:103DB3001D74FC2581F581800F7B027A0079E17DFA
:103DC300057C1C78D912081D7F027B027A0079E1F9
:103DD300129138023B977B027A0079E17D057C1CC6
:103DE30078EA12081D74069000E1F07F017B027AE5
:103DF3000079E1129138E4FCFD900110E0FEA3E0AC
:103E0300FF121491C004C005C006C0077C6F7D1269
:103E13007E837F3A12112CC004C005C006C0077B05
:103E2300027A0079E17D057C1C78C712081D74FCB9
:103E33002581F5817F027B027A0079E112913802B4
:103E43003B977B027A0079E17D057C1C78FB1208A5
:063E53001D74069000E161
:103E5900F07F017B027A0079E1129138900117E035
:103E6900FBE4C0E0C0037B027A0079E17D057C1D9B
:103E7900780C12081D158115817F027B027A007961
:103E8900E1129138023B977B027A0079E17D057C4A
:103E99001D781F12081D74069000E1F07F017B0256
:103EA9007A0079E1129138900118E0B4010E7F028D
:103EB9007B057A1D79301291380240717F027B05AA
:103EC9007A1C79D9129138023B977B027A0079E101
:103ED9007D057C1D784112081D74069000E1F07F74
:103EE900017B027A0079E112913890011EE0FEA36C
:103EF900E0FFE4FCFD121491C004C005C006C00730
:103F090074CDFC14FDFE743DFF12112C79271200AB
:103F1900F490011DE0FF129849E4FCFD121491C0D0
:103F290004C005C006C00779271200E8121288C02C
:103F390004C005C006C00790011DE0FBE4C0E0C055
:103F4900037B027A0079E17D057C1D785212081DF8
:103F590074FA2581F5817F027B027A0079E1129159
:103F690038023B977B027A0079E17D057C1D7865F3
:103F790012081D74069000E1F07F017B027A007936
:103F8900E112913890011EE0FEA3E0FFE4FCFD126E
:103F99001491C004C005C006C00774CDFC14FDFE11
:103FA900743DFF12112C79271200F47F05129849EC
:103FB900E4FCFD121491C004C005C006C0077927AE
:103FC9001200E8121288C004C005C006C00790019B
:103FD9001EE0C0E0A3E0C0E07B027A0079E17D0544
:103FE9007C1D787612081D74FA2581F5817F027B84
:103FF900027A0079E1129138023B977B027A0079C3
:10400900E17D057C1D788612081D74069000E1F09B
:104019007F017B027A0079E1129138900120E0B4A6
:10402900010D7F027B057A1D793012913880397F25
:10403900027B057A1C79D9129138023B977B027A67
:104049000079E17D057C1D789712081D74069000A2
:10405900E1F07F017B027A0079E11291387F027BDE
:0B406900057A197910129138023B977C
:07407400782BEFF21207F5B3
:10407B00129201EF792CF3792BE3B40B004003027E
:10408B0048F6FA232A904094730240B70241730218
:10409B00422F0242CD02437A024475024552024539
:0C40AB00ED02467D02476602486B80C4AF
:1040B7007F017B057A1D79A812913890010EE0C027
:1040C700E0A3E0C0E07B027A0079E17D057C1C7803
:1040D7006212081D1581158174069000E1F07F02B8
:1040E7007B027A0079E1129138792CE3B4012090B0
:1040F700010EE0B40106A3E0B4F401D3401190012E
:104107000FE024FBFB90010EE034FFF0A3EBF07906
:054117002CE3B40227B7
:07411C00900115E0B4011C45
:10412300129698E4FE7F0D1296F1E4FE7F0D900146
:104133000EE0FCA3E0FD1295CE1297191291EE2228
:10414300792CE3B4030280030248F690010EE0B435
:104153000905A3E0B4C40040030248F690010FE050
:104163002405FB90010EE03400F0A3EBF002407B4A
:104173007F017B057A1D79B9129138900109E0C05E
:10418300E0A3E0C0E07B027A0079E17D057C1C7846
:104193006212081D1581158174069000E1F07F02FB
:1041A3007B027A0079E1129138792CE3B4012090F3
:1041B3000109E0B40106A3E0B4F401D34011900176
:1041C3000AE024FBFB900109E034FFF0A3EBF07954
:0541D3002CE3B40227FB
:0741D800900115E0B4011C89
:1041DF00129698E4FE7F061296F1E4FE7F06900198
:1041EF0009E0FCA3E0FD1295CE1297191291EE2271
:1041FF00792CE3B4030280030248F6900109E0B47E
:10420F000905A3E0B4C40040030248F690010AE098
:10421F002405FB900109E03400F0A3EBF002407B92
:10422F007F017B057A1D79CA12913890011AE0FB44
:10423F00E4C0E0C0037B027A0079E17D057C1C7845
:10424F009412081D1581158174069000E1F07F020C
:10425F007B027A0079E1129138792CE3B401109046
:10426F00011AE0B41E01D3400690011AE014F07950
:05427F002CE3B402264F
:07428400900115E0B4011BDD
:10428B00129698E4FE7F0B1296F1E4FE7F0B9001E1
:10429B001AE0FD7C001295CE1297191291EE22793D
:1042AB002CE3B4030280030248F690011AE0FB7A78
:1042BB0000B4F00040030248F690011AE004F0024B
:1042CB00407B7B027A0079E17D057C1D78DB12084F
:1042DB001D7F017B027A0079E112913890010DE08C
:1042EB00FBE4C0E0C0037B027A0079E17D057C1C16
:1042FB00789412081D1581158174069000E1F07FEA
:10430B00027B027A0079E1129138792CE3B4011027
:10431B0090010DE0B41E01D3400690010DE014F0A6
:06432B00792CE3B4022628
:07433100900115E0B4011B2F
:10433800129698E4FE7F0C1296F1E4FE7F0C900131
:104348000DE0FD7C001295CE1297191291EE22799C
:104358002CE3B4030280030248F690010DE0FB7AD7
:1043680000B4F00040030248F690010DE004F002AA
:10437800407B7F017B057A1D79EC129138900113FF
:10438800E0FAA3E0FBBA0704B46C01D3503CE4FCA8
:10439800FDAE02AF03121491C004C005C006C007E9
:1043A8007C6F7D127E837F3A12112CC004C005C039
:1043B80006C0077B027A0079E17D057C1D78FD1235
:1043C800081D74FC2581F581800F7B027A0079E154
:1043D8007D057C1C78D912081D74069000E1F07FD9
:1043E800027B027A0079E1129138792CE3B401203A
:1043F800900113E0B40606A3E0B44001D340119045
:104408000114E024F6FB900113E034FFF0A3EBF075
:06441800792CE3B4022739
:07441E00900115E0B4011C40
:10442500129698E4FE7F051296F1E4FE7F05900151
:1044350013E0FCA3E0FD1295CE1297191291EE221E
:10444500792CE3B4030280030248F6900113E0B42B
:104455000705A3E0B4760040030248F6900114E096
:10446500240AFB900113E03400F0A3EBF002407B3B
:104475007F017B057A1E790E129138900110E0FEBE
:10448500A3E0FFE4FCFD121491C004C005C006C002
:10449500077C6F7D127E837F3A12112CC004C00504
:1044A500C006C0077B027A0079E17D057C1D78FD99
:1044B50012081D74FC2581F58174069000E1F07FDA
:1044C500027B027A0079E1129138792CE3B401205C
:1044D500900110E0B40106A3E0B4F401D3401190BB
:1044E5000111E024F6FB900110E034FFF0A3EBF09E
:0644F500792CE3B402275C
:0744FB00900115E0B4011C63
:10450200129698E4FE7F081296F1E4FE7F0890016D
:1045120010E0FCA3E0FD1295CE1297191291EE2243
:10452200792CE3B4030280030248F6900110E0B450
:104532000405A3E0B4B00040030248F6900111E084
:10454200240AFB900110E03400F0A3EBF002407B60
:104552007F017B057A1E791F129138900117E0FBCB
:10456200E4C0E0C0037B027A0079E17D057C1E781D
:104572003012081D1581158174069000E1F07F024A
:104582007B027A0079E1129138792CE3B401109020
:104592000117E0B40501D34006900117E014F07949
:0545A2002CE3B4022629
:0745A700900115E0B4011BB7
:1045AE00129698E4FE7F091296F1E4FE7F099001BF
:1045BE0017E0FD7C001295CE1297191291EE22791A
:1045CE002CE3B4030280030248F6900117E0B419FD
:1045DE000040030248F6900117E004F002407B7F92
:1045EE00017B057A1E7942129138900118E0B401D0
:1045FE00117B027A0079E17D057C1E785312081D2D
:10460E00800F7B027A0079E17D057C1E78641208AA
:10461E001D74069000E1F07F027B027A0079E112B0
:0D462E009138792CE364016004E3B40311BA
:10463B00900118E0B40104E4F080067401900118B5
:0C464B00F0792CE3B4020280030248F670
:07465700900115E0B4011B06
:10465E00129698E4FE7F0F1296F1E4FE7F0F900102
:10466E0018E0FD7C001295CE1297191291EE227F62
:10467E00017B057A1E797512913890011EE0FEA31A
:10468E00E0FFE4FCFD121491C004C005C006C00793
:10469E0074CDFC14FDFE743DFF12112C9000B2126D
:1046AE0000D090011DE0FF129849E4FCFD12149118
:1046BE00C004C005C006C0079000B2121285C00427
:1046CE00C005C006C00790011DE0FBE4C0E0C003BA
:1046DE007B027A0079E17D057C1D785212081D74EB
:1046EE00FA2581F58174069000E1F07F027B027A53
:1046FE000079E1129138792CE3B4011090011DE09C
:10470E00B40001D3400690011DE014F0792CE3B4FF
:02471E00022671
:07472000900115E0B4011B3C
:10472700129698E4FE7F041296F1E4FE7F0490014E
:104737001DE0FD7C001295CE1297191291EE227999
:104747002CE3B4030280030248F690011DE0B40491
:104757000040030248F690011DE004F002407B7F11
:10476700017B057A1E798612913890011EE0FEA31F
:10477700E0FFE4FCFD121491C004C005C006C007A9
:1047870074CDFC14FDFE743DFF12112C9000B21283
:1047970000D07F05129849E4FCFD121491C004C0B3
:1047A70005C006C0079000B2121285C004C005C03C
:1047B70006C00790011EE0C0E0A3E0C0E07B027ADC
:1047C7000079E17D057C1D787612081D74FA258134
:1047D700F58174069000E1F07F027B027A0079E1AF
:1047E700129138792CE3B4011E90011EE0B407063C
:1047F700A3E0B4D001D3400F90011FE014F0F49070
:0D480700011E7003E014F0792CE3B40227C9
:07481400900115E0B4011C46
:10481B00129698E4FE7F071296F1E4FE7F07900153
:10482B001EE0FCA3E0FD1295CE1297191291EE2219
:10483B00792CE3B4030280030248F690011EE0B426
:10484B000B05A3E0B4B80040030248F690011FE04B
:10485B0004F090011E60030248F6E004F002407B76
:10486B007F017B057A1E7997129138900120E0B475
:10487B0001117B027A0079E17D057C1E78531208C9
:10488B001D800F7B027A0079E17D057C1E78641216
:10489B00081D74069000E1F07F027B027A0079E13B
:0E48AB00129138792CE364016004E3B4031128
:1048B900900120E0B40104E4F08006740190012025
:0748C900F0792CE3B4022694
:0748D000900115E0B4011B8B
:1048D700129698E4FE7F0A1296F1E4FE7F0A900191
:1048E70020E0FD7C001295CE1297191291EE22025C
:0248F700407B04
:1048F9002053746172742043686172676572202065
:10490900002053746172742054726967676C652062
:1049190020002020202020202020202020202025A9
:10492900326420002053746172742044697363688F
:054939006172676500DA
:10493E00782DEEF208EFF2782FEDF28D0712507807
:10494E00EE9000C5F0A3EFF0900132E0FBE4900092
:10495E00BFF0A3EBF0E4FDFC9000B7F090011EE079
:10496E00FEA3E0FF1214919000B91200D0E4FCFDFA
:10497E009000DFE0FEA3E0FF121491C004C005C05A
:10498E0006C0077C6F7D127E837F3A12112CC00405
:10499E00C005C006C0079000D5E0FF7E00E433E4FA
:1049AE00500114FCFD12145412112CC004C005C089
:1049BE0006C0079000B9121129121495EE9000C18D
:1049CE00F0A3EFF0792FE324FD7003024C921470E4
:0F49DE0003024C9224FE6007146004146001224F
:1049ED00900120E0B40103120003792FE3FF125070
:1049FD0078EE9000BDF0A3EFF070189000BDE07060
:104A0D00129000C5E0FAA3E0FB9000BDEAF0A3EB25
:104A1D00F080109000BDE0FAA3E0FB9000C5EAF035
:104A2D00A3EBF0E4FCFD792DE3FE09E3FF121491F5
:104A3D00C004C005C006C0077C0A7DD77EA37F3C9D
:104A4D0012112C121495EE9000C3F0A3EFF0792FF4
:0E4A5D00E364066009E3B408028003024B0F15
:104A6B009000B8E0F5F0900130E065F07003024B78
:014A7B000F2B
:104A7C00E09000B8F0792FE3B406117B027A00794C
:104A8C00E17D057C4878F912081D800F7B027A00C5
:104A9C0079E17D057C49780A12081D74069000E1C5
:104AAC00F07F017B027A0079E1129138E5FEFF7EFE
:104ABC0000E4FC7D6412013DE4FC7DFF120151C059
:104ACC0006C0077B027A0079E17D057C49781B12D0
:104ADC00081D15811581792D900035E3F009A3E3AC
:104AEC00F07B027A0079E19000BDE0FCA3E0FD12BE
:104AFC0050C074259000F0F07F027B027A0079E1BF
:104B0C00129138E5FE9000B6F09000BDE0FAA3E0FB
:104B1C00FBEAFEEBFF9000C4E0FC792EE3C39CFDA6
:104B2C009000C3E0FB19E39BFCF5F0EAB5F004EF51
:104B3C00B50500500CE5FEFB7A00B4F300500205FD
:104B4C00FE9000BDE0FAA3E0FB9000C4E0FC792EDF
:104B5C00E32CFF9000C3E0FD19E33DFEF5F0EAB550
:104B6C00F005EBB50701D3400AE5FEB40001D340D4
:104B7C000215FE9000BDE0FEA3E0FF9000C4E0FA39
:104B8C00792EE3C39AFB9000C3E0FC19E39CFAF581
:104B9C00F0EEB5F004EFB50300401EA3E0F809E316
:104BAC0028FB9000C3E0F819E338FAF5F0EEB5F005
:104BBC0005EFB50301D3500122E5FEB40101D3404A
:104BCC000AE5FEFB7A00B4F20040099000BDE0FE5D
:0E4BDC00A3E0FF229000B6E0B5FE01D3401525
:104BEA009000B7E004F0B40A01D340099000BDE098
:0F4BFA00FEA3E0FF229000DEE0B40101D34049AA
:104C09001207CFE4FCFD121491C004C005C006C010
:104C190007E4FCFD9000C1E0FEA3E0FF121491C07F
:104C290004C005C006C0079000B9120089E4FEFC63
:104C3900FD743FFF12112C120FCC121522BF01096E
:104C49009000BDE0FEA3E0FF22792FE3B4070280C4
:044C5900030249ED1C
:104C5D003080032081099000BDE0FEA3E0FF22908B
:104C6D0000BFE0FCA3E0FD900132E0FB7A008AF08A
:104C7D00BC0009F5F0ED6B70030249ED9000BDE04D
:054C8D00FEA3E0FF2280
:104C9200900120E0B40103120003792FE3FF1250C8
:104CA20078EE9000BDF0A3EFF070189000BDE070B8
:104CB200129000C5E0FAA3E0FB9000BDEAF0A3EB7E
:104CC200F080109000BDE0FAA3E0FB9000C5EAF08E
:104CD200A3EBF0E4FCFD792DE3FE09E3FF1214914E
:104CE200C004C005C006C0077C0A7DD77EA37F3CF6
:104CF20012112C121495EE9000C3F0A3EFF0792F4D
:094D0200E3B403028003024D95A5
:0E4D0B009000B8E0F5F0900130E065F0607CBB
:104D1900E09000B8F07B027A0079E17D057C497862
:104D29002D12081D74069000E1F07F017B027A00C4
:104D390079E1129138E5FDFF7E00E4FC7D64120102
:104D49003DE4FC7DFF120151C006C0077B027A00D9
:104D590079E17D057C49781B12081D15811581793A
:104D69002D900035E3F009A3E3F07B027A0079E1A5
:104D79009000BDE0FCA3E0FD1250C074259000F046
:104D8900F07F027B027A0079E1129138E5FD90000B
:104D9900B6F09000BDE0FAA3E0FB9000C4E0FC7916
:104DA9002EE3C39CFD9000C3E0F819E398FCF5F0ED
:104DB900EAB5F004EBB50500500CE5FDFB7A00B44B
:104DC900F300500205FD9000BDE0FAA3E0FB90005E
:104DD900C4E0FC792EE32CFF9000C3E0FD19E33D0C
:104DE900FEF5F0EAB5F005EBB50701D3400AE5FD9C
:104DF900B40001D3400215FD9000BDE0FCA3E0FD25
:104E09009000C4E0FA792EE3C39AFB9000C3E0F85E
:104E190019E398FAF5F0ECB5F004EDB5030040227A
:104E2900ECFEEDFFA3E0F809E328FB9000C3E0FDE9
:104E390019E33DFAF5F0ECB5F005EFB50301D350F0
:104E49000122E5FDB40101D3400AE5FDFB7A00B476
:104E5900F20040099000BDE0FEA3E0FF229000B6F9
:074E6900E0B5FD01D3401587
:104E70009000B7E004F0B40A01D340099000BDE00F
:104E8000FEA3E0FF22792FE3B404028003024C92D8
:104E90003080032081099000BDE0FEA3E0FF229056
:104EA00000BFE0FCA3E0FD900132E0FB7A008AF055
:104EB000BC0009F5F0ED6B7003024C929000BDE070
:054EC000FEA3E0FF224B
:104EC5007830EEF208EFF2900132E0FBE49000CD8D
:104ED500F0A3EBF01207CFEE9000C7F0A3EFF0E4DC
:104EE500FCFD90011EE0FEA3E0FF1214919000C9A5
:034EF5001200D0D8
:104EF800900120E0B401031200031207CFEE9000E6
:104F0800D1F0A3EFF070189000D1E070129000C7B4
:104F1800E0FAA3E0FB9000D1EAF0A3EBF080109058
:104F280000D1E0FAA3E0FB9000C7EAF0A3EBF09011
:104F380000DEE064026009E064036004E0B4041E7B
:104F48009000C91200897C0A7DD77EA37F3B12118D
:104F58002C121495EE9000CFF0A3EFF0801C900077
:104F6800C91200897C0A7DD77EA37F3C12112C12BE
:104F78001495EE9000CFF0A3EFF09000D1E0FCA3E1
:104F8800E0FD9000D0E0FA7931E3C39AFB9000CFBE
:104F9800E0F819E398FAF5F0ECB5F004EDB5030084
:104FA800500CE5FEFB7A00B4F300500205FE9000B9
:104FB800D1E0FEA3E0FF9000D0E0FA7931E32AFDCA
:104FC8009000CFE0FB19E33BFCF5F0EEB5F005EF00
:104FD800B50501D3400AE5FEB40001D3400215FE31
:104FE8009000D1E0FEA3E0FF9000D0E0FA7931E331
:104FF800C39AFB9000CFE0FC19E39CFAF5F0EEB5FC
:10500800F004EFB50300401EA3E0F809E328FB9085
:1050180000CFE0F819E338FAF5F0EEB5F005EFB592
:105028000301D3500122E5FE64016006E5FE64F247
:1050380070099000D1E0FEA3E0FF223080032081B8
:10504800099000D1E0FEA3E0FF229000CDE0FCA390
:10505800E0FD900132E0FB7A008AF0BC0009F5F02F
:10506800ED6B7003024EF89000D1E0FEA3E0FF2242
:085078007832EFF2E47933F322
:105080007932E324FD601214601E24FE6005146072
:035090000E801E71
:105093007F06129849227F071298492220970F7F93
:1050A30006129849222096067F07129849227933DF
:0D50B300E304F37933E3B464C4E4FEFF22A8
:1050C0007837EBF208EAF208E9F2783AECF208ED08
:1050D000F2E4FCFD793AE3FE09E3FF121491C00407
:1050E000C005C006C007E4FCFD74C8FE7442FF1290
:1050F000112CC004C005C006C007E4FCFD7835E2F1
:10510000FE08E2FF121491121288121495EF783CF7
:10511000F27937783DE3F20908E3F20908E3F2781F
:0F5120003DE2FB08E2FA08E2F9E41200427F01E7
:10512F00793FE304F3197003E304F3793DE3FD09D9
:10513F00E3FC09E3F874011200260FBF09E2793F7F
:10514F00E304F3197003E304F3793DE3FD09E3FC92
:0C515F0009E3F87402120026E47940F322
:10516B007940E3FF7E00E4FC7D0A12013D8EF0796D
:10517B003CE3FBB2F77480B5F005EBB50701D34008
:01518B0056CD
:10518C007937E3FD09E3FC09E3F87403120026798F
:10519C0039E304F3197003E304F37940E3B4080032
:1051AC0050107937E3FD09E3FC09E3F8E41200261B
:1051BC00800F7937E3FD09E3FC09E3F8740312006F
:1051CC00267940E3B4090F7937E3FD09E3FC09E3E1
:1051DC00F874201200267940E304F37940E3B40A12
:0751EC0002800302516B2257
:1051F30075FA0075EA0075DA0075FB0075EB00754A
:10520300DB0075FC0075EC0075DC0075FD0075EDC9
:105213000075DD0075FE0075EE0075DE00C2DED29E
:0A52230093D294D295D296D297222E
:10522D00C0E0C083C082C0D0C002C003758C87753A
:0B523D008AFF900131E0B4640050468D
:10524800E004F09000D8E0FAA3E0BA0004B400014A
:10525800D3400CE014F0F49000D87003E014F09000
:065268000131E0B4325FE9
:10526E00900130E070057401F08005E4900130F09B
:10527E0090012FE004F0B40401D34043E4F0803FEA
:10528E00E4900131F0A3E004F0A3E0FAA3E0BA0049
:10529E0004B40001D3400CE014F0F4900133700319
:1052AE00E014F0900137E0FAA3E0BA0004B4000174
:1052BE00D3400CE014F0F49001377003E014F0903A
:0952CE000132E0B43B01D34010B1
:1052D700E4F0900136E004F09001357003E004F04B
:0D52E700D003D002D0D0D082D083D0E032EE
:1052F400204368617267657220526573657420206B
:10530400002066726F6D205761746368646F672153
:10531400200020202057454C434F4D4520544F201A
:1053240020200020534D41525420434841524745C8
:1053340052202000436F7079726967687420284393
:1053440029204279007777772E686F6262792D720F
:10535400632E636F6D0020496E697469616C204D22
:10536400656D6F7279200020506C656173652057FC
:105374006169742E2E2E200020202A2A20455252A4
:105384004F52202A2A2020200020204D656D6F7264
:1053940079204661696C202020004C6F6164696E3D
:1053A400672042617474657279200046726F6D20C3
:1053B4004C6F636174696F6E2025326400204C6FFA
:1053C4006164696E672044656661756C7400534D51
:1053D400415254204348415247455220425920509B
:1053E400484F454E49582400436F70797269676885
:1053F400742028432920323030362E204279205020
:10540400484F454E49582400687474703A2F2F77DA
:1054140077772E686F6262792D72632E636F6D24C5
:10542400004649524D574152452056455253494F23
:105434004E20312E313824004449534348415247C9
:10544400453A202400253364204D494E3A20240057
:1054540056424154543D25352E3266563A20240096
:1054640049424154543D25352E3266413A202400A8
:1054740050574D3D25326420202400434841524773
:10548400453A20202020240054494D45523D2534DE
:1054940064204D494E3A20240020426174746572A0
:1054A400792046756C6C792020002043686172670E
:1054B40065204465746563742120004368617267E4
:1054C40065722066756E6374696F6E00697320641B
:1054D400697361626C65642E202020200044697326
:1054E40063682E2066756E6374696F6E20002020D9
:1054F40020202025326443202534646D4168002037
:10550400204E6F204261747465727920202020003F
:10551400202025352E3266562025352E32665673C8
:105524000053544F50204449534348415247455235
:105534003F002044495343484152474520202020FE
:1055440020200020202057616974202533642073B3
:1055540065632E004449534348415247453A20422B
:105564004154544552593D2400202020203A2024FF
:105574000043415041434954593D2534646D4168C9
:105584003A20240043454C4C3D2532643A20240003
:105594004944495343483D25352E32664124002071
:1055A400537461727420446973636861726765003F
:1055B40020202020202020202020202020202020E7
:1055C40000202020202020202020252B34646D4121
:1055D400680025352E3266562025332E316641204B
:1055E400253364730025352E3266562025332E313B
:1055F4006641202533646D0025352E3266567320AE
:105604002050574D20253264200053544F502043DE
:105614004841524745523F202020002043484152F0
:1056240047452020202020202020202000434841DE
:105634005247453A20424154544552593D24004969
:105644004348415247453D25352E3266413A202490
:1056540000494D494E5F54483D2532646D413A201E
:10566400240054494D45523D2535643A20240020F8
:1056740053746172742043686172676572202000FC
:105684002054524947474C4520252B34646D4168CA
:105694000025352E326656202532646D412025338F
:1056A400646D002046554C4C5920434841524745AF
:1056B4002020200020444953434841524745204478
:1056C4004F4E4520002055534552205445524D49D4
:1056D4004E415445440020424154542E204F5645D7
:1056E400522D564F4C5400204241545420444953A7
:0856F400434F4E4E45435400A4
:1056FC00204C4F5720535550504C5920564F4C541A
:10570C00002044495343482E2020252B34646D41FE
:10571C0068002044495343482E54494D45202533B5
:10572C00646D00204348415247452020252B3464AA
:10573C006D416800204348472E54494D4520202098
:10574C002533646D00204D4554484F443A20434363
:10575C002D4356202000204D4554484F443A204EAE
:10576C0045472D64562000204D4554484F443A205F
:10577C00494E464C45582000204D4554484F443A1C
:10578C002054494D4552202000204D4554484F444B
:10579C003A205A45524F2D6456002025352E32663C
:1057AC0056702025352E32665665200020535550F4
:1057BC00504C59202025352E32665673200020205F
:0F57CC00204E6F202020202059657320202000C0
:1057DB007580FF7590FF75A0FF75B0FFE4FE7FFA33
:1057EB001291D61290051207F5E4FF1290F9758904
:1057FB0021758C87758AFF75985253877F758DFB42
:10580B00D28CD28E75A8921207EB1251F31295C55A
:09581B0030C23A900120E0603433
:1058240012026C7F017B057A5279F41291387F025F
:105834007B057A537905129138C2B43080143081D3
:015844001152
:1058450020B40312919A7E017FF41291D6B2B480EE
:10585500E9D2B4308007208104D2008002C2007FE3
:10586500017B057A5379161291387F027B057A53AD
:1058750079271291387E077FD01291D67F017B055B
:105885007A5379381291387F027B057A5379491218
:1058950091387E037FE81291D6740190010CF09047
:1058A5000116F090011CF07404A3F0900113740725
:1058B500F0A37476F09001097404F0A374B0F0902D
:1058C500011E7408F0A37484F09001107403F0A312
:1058D50074E8F0740F900117F07401900120F074D2
:1058E5003C90011AF090010DF0A37404F0A374B07C
:1058F500F0E4FFFE900112F0900118F0A3F0900182
:105905001BF0129607BE01028003025A0EBF000269
:055915008003025A0EA0
:10591A007401900115F0E4FE7F01129607EF9001E1
:10592A000CF0E4FE7F02129607EF900146F0540F46
:10593A00900116F0900146E05480B40800E440015A
:10594A0004900119F0900146E05440B40700E44085
:10595A00010490011BF0E4FE7F03129607EF900109
:10596A001CF0E4FE7F04129607EF90011DF0E4FE9E
:10597A007F05129607EE900113F0A3EFF0E4FE7F85
:10598A0006129607EE900109F0A3EFF0E4FE7F07F6
:10599A00129607EE90011EF0A3EFF0E4FE7F0812C4
:1059AA009607EE900110F0A3EFF0E4FE7F0912963D
:1059BA0007EF900117F0E4FE7F0A129607EF9001B5
:1059CA0020F0E4FE7F0B129607EF90011AF0E4FE36
:1059DA007F0C129607EF90010DF0E4FE7F0D1296F0
:1059EA0007EE90010EF0A3EFF0E4FE7F0E12960789
:1059FA00EF900112F0E4FE7F0F129607EF90011864
:045A0A00F0025B95B6
:105A0E007F017B057A53795A1291387F027B057A92
:105A1E0053796B129138129698E4FE7F0A1291D642
:105A2E00E4FEFF1296F1E4FDFEFF7C011295CE120C
:105A3E009719E4FEFF129607BE01028003025B6611
:085A4E00BF00028003025B6649
:105A56007401900115F0129698E4FE7F0A1291D611
:105A6600E4FE7F0190010CE0FD7C001295CE9001D2
:105A760016E0900146F0900119E0B4010790014646
:105A8600E04480F090011BE0B40107900146E04439
:105A960040F0E4FE7F02900146E0FD7C001295CEC8
:105AA600E4FE7F0390011CE0FD7C001295CEE4FE2F
:105AB6007F0490011DE0FD7C001295CEE4FE7F057B
:105AC600900113E0FCA3E0FD1295CEE4FE7F069064
:105AD6000109E0FCA3E0FD1295CEE4FE7F079001EC
:105AE6001EE0FCA3E0FD1295CEE4FE7F08900110B7
:105AF600E0FCA3E0FD1295CEE4FE7F09900117E0DD
:105B0600FD7C001295CEE4FE7F0A900120E0FD7C2C
:105B1600001295CEE4FE7F0B90011AE0FD7C001288
:105B260095CEE4FE7F0C90010DE0FD7C001295CE33
:105B3600E4FE7F0D90010EE0FCA3E0FD1295CEE49D
:105B4600FE7F0E900112E0FD7C001295CEE4FE7FF2
:105B56000F900118E0FD7C001295CE129719802F48
:105B6600E4900115F07F017B057A53797C12913818
:105B76007F027B057A53798D1291381291EEE4FEFD
:105B86007FC81291D61291EE7E027FBC1291D61278
:0B5B96008D6230800C20810930000679
:105BA1001291EE123B56900115E0B40102800302FE
:025BB1005DC9CC
:105BB300900112E0B401005003025D21E0B40A0138
:065BC300D34003025D2146
:105BC900E0FB24FFFFE434FFFEE4FC7D0A12013D03
:105BD900EF2410FFE43E9001A6F0A3EFF0EB2400C0
:105BE900FBE43455FAC002C0039001A6E0FEA3E02D
:105BF900FF129607D005D0F0EEB5F0028003025CE3
:0A5C0900D9EFB505028003025CD953
:105C13007F017B057A53799E129138900112E0FB44
:105C2300E4C0E0C0037B027A0079E17D057C537810
:105C3300AF12081D158115817F027B027A0079E17D
:105C43001291389001A7E02401FF9001A6E03400EF
:105C5300FE129607EF9000DEF09001A7E02402FF0A
:105C63009001A6E03400FE129607EE9000D3F0A355
:105C7300EFF09001A7E02403FF9001A6E03400FEBB
:105C8300129607EF9000D5F09001A7E02404FF904F
:105C930001A6E03400FE129607EE9000DAF0A3EFBF
:105CA300F09001A7E02405FF9001A6E03400FE1266
:105CB3009607EE9000DCF0A3EFF09001A7E0240636
:105CC300FF9001A6E03400FE129607EE9000DFF08D
:065CD300A3EFF0025DC921
:105CD9007F017B057A5379C11291387F027B057A5E
:105CE90053796B129138E49000DEF09000D374037D
:105CF900F0A374E8F07408A3F09000DA7403F0A339
:105D090074E8F0A37401F0A374F4F09000DF740553
:085D1900F0A37478F0025DC9EB
:105D21007F017B057A5379C11291387F027B057A15
:105D310053796B129138E4FE7F10129607BE5559C4
:035D4100BF015649
:105D4400E4FE7F11129607EF9000DEF0E4FE7F126E
:105D5400129607EE9000D3F0A3EFF0E4FE7F131247
:105D64009607EF9000D5F0E4FE7F14129607EE90AC
:105D740000DAF0A3EFF0E4FE7F15129607EE900030
:105D8400DCF0A3EFF0E4FE7F16129607EE9000DF3E
:065D9400F0A3EFF0802FE8
:105D9A00E49000DEF09000D37403F0A374E8F0748A
:105DAA0008A3F09000DA7403F0A374E8F0A3740176
:105DBA00F0A374F4F09000DF7405F0A37478F09007
:105DCA0000DEE0B40101D340067402900116F0E44B
:105DDA00900131F0900135F0A3F0900132F0D2A990
:105DEA00128FD29000D6E4F0A3F00490010BF0C217
:105DFA000190014FF0E4FDFC900152F0900109E09E
:105E0A00FEA3E0FF121491C004C005C006C0077CBF
:105E1A006F7D127E837F3A12112C9001391200D0C5
:105E2A00E4FCFD90010EE0FEA3E0FF121491C00411
:105E3A00C005C006C0077C6F7D127E837F3A1211AF
:105E4A002C90013D1200D0E4FCFD90011EE0FEA35F
:105E5A00E0FF121491C004C005C006C00774CDFC4F
:105E6A0014FDFE743DFF12112C9001411200D075F1
:105E7A00FD7F75ED7F75DD42D2DE7E037FE81291EC
:105E8A00D61251F31291EE1207F5900120E0B401F7
:0E5E9A0003120262900118E0B40001D34065CB
:105EA8007F0D12926A7F0A12926A7F0A12926A7BA7
:105EB800057A5379D21292797F0D12926A7F0A126B
:105EC800926A7B057A5379EC1292797F0D12926A65
:105ED8007F0A12926A7F0A12926A7B057A54790CB9
:105EE8001292797F0D12926A7F0A12926A7F0A12C1
:105EF800926A7B057A5479251292797F0D12926AFB
:055F08007F0A12926AFD
:105F0D0090014EE0FB7A008AF0900135E0FCA3E0B1
:105F1D00FDBC00088BF06B7003026163900118E00B
:095F2D00B40001D35003026163CA
:0F5F3600ED90014EF0A3E0B40402800302604E30
:105F45007F0D12926A7F0A12926A7B057A54793C18
:105F5500129279900135E0C0E0A3E0C0E07B027ABF
:105F65000079E17D057C54784912081D158115815C
:105F75007B027A0079E1129279E4FCFD90015AE006
:105F8500FEA3E0FF121491C004C005C006C007902F
:105F95000141121285C004C005C006C0077B027A04
:105FA5000079E17D057C54785412081D74FC258127
:105FB500F5817B027A0079E1129279E4FCFD90018A
:105FC50054E0FEA3E0FF121491C004C005C006C052
:105FD50007900139121285C004C005C006C0077CB0
:105FE5006F7D127E837F3A12112CC004C005C00656
:105FF500C0077B027A0079E17D057C54786412083C
:106005001D74FC2581F5817B027A0079E112927974
:10601500E5FDFF7E00E4FC7D6412013DE4FC7DFFAF
:10602500120151C006C0077B027A0079E17D057C2B
:1060350054787412081D1581158174259000E7F0B8
:106045007B027A0079E112927990014FE0B4070260
:056055008003026163FD
:10605A007F0D12926A7F0A12926A7B057A54797FBF
:10606A00129279900137E0C0E0A3E0C0E07B027AA7
:10607A000079E17D057C54788C12081D1581158103
:10608A007B027A0079E1129279E4FCFD90015AE0F0
:10609A00FEA3E0FF121491C004C005C006C0079019
:1060AA000141121285C004C005C006C0077B027AEE
:1060BA000079E17D057C54785412081D74FC258111
:1060CA00F5817B027A0079E1129279E4FCFD900174
:1060DA0054E0FEA3E0FF121491C004C005C006C03C
:1060EA0007900139121285C004C005C006C0077C9A
:1060FA006F7D127E837F3A12112CC004C005C00640
:10610A00C0077B027A0079E17D057C547864120825
:10611A001D74FC2581F5817B027A0079E11292795E
:10612A00E5FEFF7E00E4FC7D6412013DE4FC7DFF98
:10613A00120151C006C0077B027A0079E17D057C15
:10614A0054787412081D1581158174259000E7F0A2
:10615A007B027A0079E1129279900120E0B401037E
:10616A00120003129201EF90014CF090014FE0B43B
:10617A000503026F835014E014602814700302654B
:10618A00AD24FE700302692D028D5FE024F97003CD
:10619A000277E324FE70030286D6147003028AA0F3
:0361AA00025F0D84
:1061AD00D2B2D2B3D2B490014CE0B401028003025A
:0861BD0062AA2001030262AA9C
:0B61C500900116E06403700302628288
:1061D0009000DEE06009E0B40102800302625AE44C
:1061E000FCFD90015AE0FEA3E0FF121491C004C030
:1061F00005C006C007900141121285C004C005C049
:1062000006C0079000D5E0FB7A00E433E4500114A7
:10621000FCFDAE02AF03121454121288C004C00574
:10622000C006C0077CCD7DCC7EAC7F3F121522BF5F
:02623000012843
:10623200C2B41291C37F017B057A54799D129138C1
:106242007F027B057A5479AE1291381291EE7E0765
:086252007FD01291D6025F0D0E
:10625A00740190010BF0740590014FF0128FD290E7
:10626A00011AE0FBE4900133F0A3EBF0A3E4F0A3FE
:08627A00F0900132F0025F0D0B
:10628200C2B41291C37F017B057A5479BF1291384F
:106292007F027B057A5479D01291381291EE7E07F3
:0F62A2007FD01291D6025F0D90014CE0B402093B
:1062B100120269123A0012000690014CE0B4035335
:0362C10030015059
:0862C400900116E06402602263
:1062CC00740290014FF0128FD290011AE0FBE4900F
:1062DC000133F0A3EBF0A3E4F0A3F0900132F00251
:0262EC008D5FC4
:1062EE001291C37F017B057A5479E11291387F02B6
:1062FE007B057A5479D01291381291EE7E077FD0B9
:10630E001291D6025F0D7F05129849EE90015AF058
:0F631E00A3EFF090010CE0B40102800302648B46
:10632D009000DEE0FAB403030263F3500CEA601A46
:10633D0014601714606202648BEA24FC700302631C
:0A634D00F314700302644002648B35
:10635700E4FCFD90015AE0FEA3E0FF121491C00493
:10636700C005C006C007900141121285C004C005D0
:10637700C006C0077CF57DBE7E207F4012112CC071
:1063870004C005C006C00774ABFC14FDFE743EFFD5
:1063970012112C121495EF9000D5F002648BE4FCD7
:1063A700FD90015AE0FEA3E0FF121491C004C0055E
:1063B700C006C007900141121285C004C005C0067F
:1063C700C0077CB07DDE7E687F3F12112CC004C001
:1063D70005C006C00774ABFC14FDFE743EFF121126
:1063E7002C121495EF9000D5F002648BE4FCFD901D
:1063F700015AE0FEA3E0FF121491C004C005C006D5
:10640700C007900141121285C004C005C006C0072D
:106417007C4D7D187E807F3F12112CC004C005C0C3
:1064270006C00774ABFC14FDFE743EFF12112C125C
:106437001495EF9000D5F0804BE4FCFD90015AE0F5
:10644700FEA3E0FF121491C004C005C006C0079068
:106457000141121285C004C005C006C0077C207D1B
:10646700527EC07F3F12112CC004C005C006C00772
:1064770074ABFC14FDFE743EFF12112C121495EF41
:106487009000D5F09000D3E0C0E0A3E0C0E0A3E027
:10649700FBE4C0E0C0037B027A0079E17D057C5410
:1064A70078F212081D74FC2581F5819000D5E07003
:1064B7000674419000E7F07B027A0079E19000DEF4
:1064C700E0FD128F8E7F017B027A0079E11291380D
:1064D70090011DE0FF129849EE9001A8F0A3EFF09C
:1064E700E4FCFD90015AE0FEA3E0FF121491C00402
:1064F700C005C006C007900141121285C004C0053F
:10650700C006C0077466FEFCFD743FFF121522BF6C
:0A651700FF0280069000D5E0701925
:106521007B027A0079E17D057C55780312081D74A0
:09653100069000E1F0C201806552
:10653A00E4FCFD9001A8E0FEA3E0FF121491C00460
:10654A00C005C006C007900141121285C004C005EB
:10655A00C006C007E4FCFD90015AE0FEA3E0FF126A
:10656A001491C004C005C006C007900141121285EB
:10657A00C004C005C006C0077B027A0079E17D0528
:10658A007C55781412081D74F82581F581740290DF
:10659A0000E1F0D2017F027B027A0079E1129138A0
:1065AA00025F0DD2B3D2B41251F37F05129849E4B7
:1065BA00FCFD121491C004C005C006C00790014139
:1065CA00121285C004C005C006C0077466FEFCFD31
:0965DA00743FFF121522BFFF4AB5
:1065E300C201E4900149F0740A90014FF0E4900174
:1065F30051F07404900150F01291EE1251F3128F86
:10660300D27F05129849EE900129F0A3EFF0900193
:106613001DE0FF129849EE90012DF0A3EFF09001D9
:1066230033E4F0A37404F0025F0D90014CE0B40373
:0F66330007900133E4F0A3F090014CE0B402595A
:106642007B057A557925128E97EF64016003028DDE
:016652005FE8
:106653007F05129849EE900129F0A3EFF01251F350
:106663001291EEE4900149F0740A90014FF0E49026
:106673000151F07402900150F0128FD290011DE08D
:10668300FF129849EE90012DF0A3EFF0900133E44F
:10669300F0A37404F0025F0D7B027A0079E17D05BB
:1066A3007C55783612081D7B027A0079EC9000DE67
:1066B300E0FD128F8E74069000E1F07F017B027A79
:1066C3000079E1129138900133E0C0E0A3E0C0E02B
:1066D3007B027A0079E17D057C55784712081D1508
:1066E30081158174029000E1F0900130E0B4010A59
:0A66F30074079000E2F0C2B28002CA
:1066FD00D2B27F027B027A0079E112913890013398
:0D670D00E0600302691FA3E0600302691F42
:0D671A00900118E0B40001D3500302680C98
:106727007F0D12926A7F0A12926A7B027A0079E1E0
:106737007D057C55785812081D7B027A0079E11295
:1067470092797B027A0079E17D057C55786D120894
:106757001D7B027A0079E19000DEE0FD128F8E7BCF
:10676700027A0079E11292799000D3E0C0E0A3E0C9
:10677700C0E07B027A0079E17D057C5578751208C7
:106787001D158115817B027A0079E11292799000BB
:10679700D5E0FDE4C0E0C0057B027A0079E17D0524
:1067A7007C55788812081D158115817B027A00793E
:1067B700E11292799000DCE0FEA3E0FFE4FCFD1219
:1067C7001491C004C005C006C0077C6F7D127E838C
:1067D7007F3A12112CC004C005C006C0077B027A9D
:1067E7000079E17D057C55789412081D74FC25819C
:1067F700F5817B027A0079E11292797F0D12926A14
:106807007F0A12926AC2B275FD0175ED0175DD420C
:10681700D2DE90013D120089E4FCFD9000DCE0FE31
:10682700A3E0FF12149112112C121495EE90015649
:10683700F0A3EFF09000D6E4F0A3F0C0E0C0E0745E
:1068470061C0E07445C0E09000DAE0FEA3E0FFE439
:10685700FCFD121491121288C004C005C006C007BF
:10686700E4FCFD74C8FE7442FF12112C121495EE5D
:106877009000D8F0A3EFF07B027A0079E17D057CE8
:106887005578A312081D74069000E1F07F017B0282
:106897007A0079E11291387F027B057A5579B41233
:1068A70091387F011290F9900156E0FEA3E0FF7D39
:1068B7000312493EEE900154F0A3EFF07F027B05EF
:1068C7007A5579B4129138E4FF1290F97404900163
:0B68D7004FF0E4900152F090014BF0F4
:1068E200900154E0FCA3E0FD90014BE0FA2AFB2466
:1068F2006AF582E43401F583ECF0A3EDF090015ADD
:10690200E0FCA3E0FDEB247EF582E43401F583ECA8
:10691200F0A3EDF090014BE004F0B40AC39001350E
:10692200E4F0A3F0900132F0025F0DC2B290014C8C
:10693200E064016004E0B403067405900152F09033
:0969420000D8E0705DA3E070597B
:10694B009000D7E004F09000D67003E004F0E4C0B0
:10695B00E0C0E07461C0E07445C0E0E4FCFD900170
:10696B0054E0FEA3E0FF121491C004C005C006C0A2
:10697B000790013D121285121288C004C005C00693
:10698B00C007E4FCFD74C8FE7442FF12112C1214F4
:10699B0095EE9000D8F0A3EFF090014CE0B40279A3
:1069AB007B057A557925128E97EF64016003028D72
:0169BB005F7C
:1069BC007F05129849EE900129F0A3EFF01251F3E4
:1069CC001291EEE4900149F0740A90014FF0E490BA
:1069DC000151F07402900150F09000D6E0FAA3E05F
:1069EC00FB900125EAF0A3EBF0900135E0FAA3E06F
:1069FC002401FBE43A900127F0A3EBF090011DE099
:106A0C00FF129849EE90012DF0A3EFF0900133E4C2
:106A1C00F0A37404F0025F0D900132E0F5F09001E8
:096A2C004DE065F07003026BE619
:106A3500900152E0B40001D34003E014F090011D31
:106A4500E0FF129849EE9001A8F0A3EFF07F041241
:106A55005078EE90017AF0A3EFF09001AE120100AC
:096A650000000000E490014BF078
:106A6E0090014BE025E0246CF582E43401F583E0DF
:106A7E00FCA3E0FD90014BE0FA2AFF246AF582E4C4
:106A8E003401F583ECF0A3EDF09001AE120089EF26
:106A9E00246AF582E43401F583E0FEA3E0FFE4FC12
:106AAE00FD1201289001AE1200D090014BE004F0CF
:106ABE00B408AD75F0039001AE1200C412000E9032
:106ACE000154EEF0A3EFF0A3E0FEA3E0FFE4FCFD23
:106ADE00121491C004C005C006C0077C0A7DD77E83
:106AEE00A37F3C12112C121495EE900166F0A3EFC9
:106AFE00F0900154E0FCA3E0FDA3E0FAA3E0FB90CC
:106B0E000167E0F8EBC398FB900166E0F8EA98FAAB
:106B1E00F5F0ECB5F004EDB50300401EE0FAA3E08D
:106B2E00FB900157E02BFB900156E03AFAF5F0ECA2
:0A6B3E00B5F005EDB50301D34015D5
:106B4800900156E0FEA3E0FF7D0412493EEE90015D
:106B580054F0A3EFF01207CFEE90018EF0A3EFF000
:0F6B68009001AE12010000000000E490014BF01C
:106B770090014BE025E02480F582E43401F583E0C1
:106B8700FCA3E0FD90014BE0FA2AFF247EF582E4A6
:106B97003401F583ECF0A3EDF09001AE120089EF1C
:106BA700247EF582E43401F583E0FEA3E0FFE4FCF4
:106BB700FD1201289001AE1200D090014BE004F0C5
:106BC700B408AD75F0039001AE1200C412000E9028
:106BD700015AEEF0A3EFF0900132E090014DF090F2
:106BE700015AE0B40006A3E0B40001D35003026CDD
:106BF700F7E4FCFD90015AE0FEA3E0FF121491C0F8
:106C070004C005C006C007900141121285C004C028
:106C170005C006C0079000D5E0FB7A00E433E450D6
:106C27000114FCFDAE02AF03121454C004C005C02A
:106C370006C007E4FCFD900110E0FEA3E0FF12147C
:106C470091C004C005C006C0077C6F7D127E837F9C
:106C57003A12112C12112C121522BFFF02800302C7
:026C67006CF7C8
:106C690090015AE0FAA3E0FB900129EAF0A3EBF0C6
:106C79001251F39000D6E0FAA3E0FB900125EAF067
:106C8900A3EBF0900135E0FAA3E02401FBE43A908C
:106C99000127F0A3EBF090011DE0FF129849EE9057
:0D6CA900012DF0A3EFF0900116E0B4011DE5
:106CB60090010DE0FBE4900133F0A3EBF074059036
:0D6CC600014FF0900135E4F0A3F0028D5F66
:106CD3001291EEE4900149F0740A90014FF0E490B0
:106CE3000151F004900150F0900133E4F0A37404D7
:106CF300F0025F0DE4FCFD90015AE0FEA3E0FF12F9
:106D03001491C004C005C006C0079001411212854A
:106D1300C004C005C006C0077466FEFCFD743FFFD7
:066D2300121522BFFF6BF8
:106D29001291EE1251F3E4900149F0740A90014F67
:106D3900F0E4900151F07404900150F09000D6E015
:106D4900FAA3E0FB900125EAF0A3EBF0900135E00E
:106D5900FAA3E02401FBE43A900127F0A3EBF090B9
:106D6900015AE0FAA3E0FB900129EAF0A3EBF090C5
:106D7900011DE0FF129849EE90012DF0A3EFF0906C
:106D89000133E4F0A37404F0025F0D9000D6E0FA39
:106D9900A3E0F4FBEAF4FA0BEB70010AC002C003AA
:106DA9007B027A0079E17D057C5578C512081D15AD
:106DB90081158190010BE06401600A9000DEE0B466
:056DC9000101D34010A0
:106DCE007B027A0079E39000DEE0FD128F8E801751
:106DDE0074449000E4F014A3F0743AA3F090010B05
:106DEE00E024309000E7F090012FE0FA7404C39A8B
:106DFE009000E1F07406A3F07F017B027A0079E146
:0C6E0E00129138900152E06003026F1FE7
:106E1A00900135E06003026EA3A3E0707C9001321A
:106E2A00E0FBE4C0E0C003FCFD900154E0FEA3E0F7
:106E3A00FF121491C004C005C006C00790013D129C
:106E4A001285C004C005C006C0077C6F7D127E8310
:106E5A007F3A12112CC004C005C006C007E4FCFD2D
:106E6A0090015AE0FEA3E0FF121491C004C005C0CD
:106E7A0006C007900141121285C004C005C006C0B1
:106E8A00077B027A0079E17D057C5578D612081DC8
:106E9A0074F62581F581026F75900135E0C0E0A393
:106EAA00E0C0E0E4FCFD900154E0FEA3E0FF121410
:106EBA0091C004C005C006C00790013D121285C0EA
:106ECA0004C005C006C0077C6F7D127E837F3A121C
:106EDA00112CC004C005C006C007E4FCFD90015A8D
:106EEA00E0FEA3E0FF121491C004C005C006C0076B
:106EFA00900141121285C004C005C006C0077B027A
:106F0A007A0079E17D057C5578E912081D74F62529
:056F1A0081F5818056A5
:106F1F00E5FDFF7E00E4FC7D6412013DE4FC7DFF96
:106F2F00120151C006C007E4FCFD9001A8E0FEA3CA
:106F3F00E0FF121491C004C005C006C007900141C4
:106F4F00121285C004C005C006C0077B027A007903
:106F5F00E17D057C5578FC12081D74FA2581F581B9
:106F6F0074259000F0F07F027B027A0079E1129194
:106F7F0038025F0DD2B2D2B41251F37F0512984985
:106F8F00E4FCFD121491C004C005C006C0079001B7
:106F9F0041121285C004C005C006C0077466FEFC0E
:0A6FAF00FD743FFF121522BFFF4AD8
:106FB9001291EE1251F3C201E4900149F0740A9062
:106FC900014FF0E4900151F07404900150F09001E8
:106FD9005AE0FAA3E0FB900129EAF0A3EBF0900153
:106FE9001DE0FF129849EE90012DF0A3EFF09001FA
:106FF90033E4F0A37404F0025F0D90014CE0B40196
:0F70090007900133E4F0A3F090014CE0B402567D
:107018007B057A56790E128E97EF64016003028D14
:017028005F08
:107029007F05129849EE900129F0A3EFF090011D18
:10703900E0FF129849EE90012DF0A3EFF01251F301
:107049001291EEE4900149F0740A90014FF0E49036
:107059000151F07402900150F0900133E4F0A374EF
:1070690004F0025F0D7B027A0079E17D057C567898
:107079001F12081D7B027A0079E99000DEE0FD12FB
:107089008F8E74069000E1F07F017B027A0079E12E
:10709900129138900133E0C0E0A3E0C0E07B027AAE
:1070A9000079E17D057C55784712081D1581158108
:0D70B90074029000E1F0900130E0B4010A93
:0A70C60074079000E2F0C2B38002EC
:1070D000D2B37F027B027A0079E1129138900133BA
:0D70E000E0600302777BA3E0600302777B92
:1070ED00900139120089E4FCFD74A0FE7441FF1279
:1070FD00112C121495EE90015EF0A3EFF090011398
:10710D00E0FEA3E0FFE4FCFD121491C004C005C035
:10711D0006C0077C6F7D127E837F3A12112CC0044E
:10712D00C005C006C0079000D5E0FD7C00E4C0E0BE
:10713D00EDFFD0E0FE33E4500114FDFC12145412A7
:10714D00112CC004C005C006C007900141121129C1
:10715D00121495EE900162F0A3EFF09000DEE07056
:10716D005F900117E0FF7E00E433E4500114FCFD55
:10717D00121454C004C005C006C0077C6F7D127E7A
:10718D00837F3A12112CC004C005C006C0079001C0
:10719D0041121129C004C005C006C0079000D5E0FA
:1071AD00FD7C00E4C0E0EDFFD0E0FE33E4500114BF
:1071BD00FDFC12145412112C121495EF900145F090
:1071CD009000DFE0FEA3E0FFE4FCFD121491C0048B
:1071DD00C005C006C0077C6F7D127E837F3A1211F9
:1071ED002CC004C005C006C0079000D5E0FFE4FE2A
:1071FD0033E4500114FDFC12145412112CC004C0C0
:10720D0005C006C007900141121129121495EE9088
:10721D000158F0A3EFF09000D3E0FEA3E0FFE4FCF3
:10722D00FD121491C004C005C006C007E4FCFD7436
:10723D0080FE743FFF12112CC004C005C006C007AC
:10724D009000DAE0FEA3E0FFE4FCFD1214911212AF
:10725D0088C004C005C006C007E4FCFD7461FE745F
:10726D0045FF12112C121495EE900137F0A3EFF09B
:10727D009000D5E0FF7E00E433E4500114FCFD12D4
:10728D001454C004C005C006C0077CEC7D517EB807
:10729D007F3F12112CC004C005C006C007900141EC
:1072AD00121129121495EE900164F0A3EFF09001E4
:1072BD0041120089E4FEFCFD743FFF12112C1214E3
:1072CD0095EE900168F0A3EFF090011DE0B4046D10
:1072DD00E4FCFD9000DFE0FEA3E0FF121491C0047A
:1072ED00C005C006C0077C6F7D127E837F3A1211E8
:1072FD002CC004C005C006C0079000D5E0FF7E007D
:10730D00E433E4500114FCFD12145412112CC0048A
:10731D00C005C006C007E4FCFD74C0FE743FFF123B
:10732D000FD5C004C005C006C00790014112112938
:10733D00121495EE90015CF0A3EFF0801D900141C9
:10734D00120089E4FCFD7428FE7441FF12112C1209
:10735D001495EE90015CF0A3EFF09000DEE0FA647E
:10736D00026009EA64036004EAB4042D9001391245
:10737D0000899000D5E0FF7E00E4FC7D5012013DB8
:10738D00EE33E4500114FDFC12145412112C12149E
:10739D0095EE900160F0A3EFF09000DEE0B4053AB9
:1073AD009000D3E0FEA3E0FFE4FCFD121491C004B5
:1073BD00C005C006C0077C297D5C7E8F7F3D121104
:1073CD002CC004C005C006C0079001391211291246
:1073DD001495EE900160F0A3EFF09000DEE0B401A3
:1073ED0001D3404BE4FCFD900160E0FEA3E0FF12F1
:1073FD001491C004C005C006C00790013912008960
:10740D00E4FCFD74A0FE7442FF12112C121522BF74
:10741D00FF1D900139120089E4FCFD74A0FE744239
:10742D00FF12112C121495EE900160F0A3EFF09065
:10743D0000DEE0B40101D34006740190010BF0E4CD
:10744D00900147F0A3F0C20290014AF0900152F072
:10745D007960F309F37962F309F3A3F0900118E071
:03746D00B4000167
:06747000D350030275A7D2
:107476007F0D12926A7F0A12926A7B027A0079E184
:107486007D057C56783112081D7B027A0079E1125F
:1074960092797B027A0079E17D057C55786D120838
:1074A6001D7B027A0079E19000DEE0FD128F8E7B73
:1074B600027A0079E11292799000D3E0C0E0A3E06D
:1074C600C0E07B027A0079E17D057C55787512086B
:1074D6001D158115817B027A0079E112927990005F
:1074E600D5E0FBE4C0E0C0037B027A0079E17D05CC
:1074F6007C55788812081D158115817B027A0079E2
:10750600E11292799000DAE0FEA3E0FFE4FCFD12BE
:107516001491C004C005C006C0077C6F7D127E832F
:107526007F3A12112CC004C005C006C0077B027A40
:107536000079E17D057C56784312081D74FC25818F
:10754600F5817B027A0079E1129279900160E0C0C0
:10755600E0A3E0C0E07B027A0079E17D057C567805
:107566005512081D158115817B027A0079E1129268
:1075760079900137E0C0E0A3E0C0E07B027A0079B1
:10758600E17D057C56786612081D158115817B0202
:107596007A0079E11292797F0D12926A7F0A12922D
:1075A6006A9000D6E4F0A3F0C0E0C0E07461C0E0E9
:1075B6007445C0E09000DAE0FEA3E0FFE4FCFD12B3
:1075C6001491121288C004C005C006C007E4FCFD71
:1075D60074C8FE7442FF12112C121495EE9000D856
:1075E600F0A3EFF0C2B375FE0175EE0175DE42D26F
:1075F600DEC2039001391200899000DAE0FEA3E0B2
:10760600FFE4FCFD12149112112C121495EE900158
:1076160056F0A3EFF0900139120089E4FCFD74489E
:10762600FE7442FF12112C121495EE9001AAF0A3DB
:10763600EFF09000D3E0FEA3E0FFE4FCFD1214910E
:10764600C004C005C006C0077CCD7DCC7E4C7F3D06
:1076560012112CC004C005C006C0079001391211D2
:1076660029121495EE9001ACF0A3EFF0E4FCFD9026
:1076760001ACE0FEA3E0FF121491C004C005C006F1
:10768600C007900139121285C004C005C006C007A4
:10769600E4FCFD74A0FE7441FF121522BFFF1D908D
:1076A6000139120089E4FCFD74A0FE7441FF121139
:1076B6002C121495EE9001ACF0A3EFF07B027A0049
:1076C60079E17D057C56787312081D74069000E1F9
:1076D600F07F017B027A0079E11291387F027B0507
:1076E6007A5579B41291387F011290F9900156E0DB
:1076F600FEA3E0FF7D0612493EEE900154F0A3EF93
:10770600F07F027B057A5579B4129138E4FF129026
:05771600F9E490014BB5
:01771B00F07D
:10771C00900154E0FCA3E0FD90014BE0FA2AFB241D
:10772C006AF582E43401F583ECF0A3EDF090015A94
:10773C00E0FCA3E0FDEB247EF582E43401F583EC60
:10774C00F0A3EDF090011DE0FF12984990014BE081
:10775C00FA2A2492F582E43401F583EEF0A3EFF0DB
:10776C0090014BE004F0B40AA7740790014FF0901D
:10777C0000D3E0FEA3E0FFE4FCFD121491C004C0B2
:10778C0005C006C007E4FCFD7480FE743FFF1211B7
:10779C002CC004C005C006C007E4FCFD9000DAE074
:1077AC00FEA3E0FF121491121288C004C005C0069B
:1077BC00C007E4FCFD7461FE7445FF12112C121419
:1077CC0095EE900137F0A3EFF0900135E4F0A3F0C3
:1077DC00900132F0025F0DC2B390014CE064016085
:1077EC0004E0B403067405900152F09000D8E070E8
:0577FC005DA3E07059DF
:107801009000D7E004F09000D67003E004F0E4C0EB
:10781100E0C0E07461C0E07445C0E0E4FCFD9001AB
:1078210054E0FEA3E0FF121491C004C005C006C0DD
:1078310007900139121285121288C004C005C006D2
:10784100C007E4FCFD74C8FE7442FF12112C12142F
:1078510095EE9000D8F0A3EFF0900137E07004A30B
:10786100E060199000D3E0FAF5F0A3E0FB9000D6B8
:0C787100E0B5F006A3E0B50301D34070C1
:10787D001251F31291EE7403900149F0740A9001C4
:10788D004FF0E4900151F0900150F09000D6E0FAE5
:10789D00A3E0FB900121EAF0A3EBF0900135E0FAB3
:1078AD00A3E02401FBE43A900123F0A3EBF0900157
:1078BD005AE0FAA3E0FB900129EAF0A3EBF079621C
:1078CD00A3E3F009A3E3F090011DE0FF129849EE48
:1078DD0090012DF0A3EFF0900133E4F0A37404F0C8
:0C78ED0090014CE0B4020280030279819B
:0E78F9007B057A56790E128E97EF6401707A35
:107907001251F31291EE740190010BF0E4900149CA
:10791700F0740A90014FF0E4900151F07402900165
:1079270050F09000D6E0FAA3E0FB900121EAF0A323
:10793700EBF0900135E0FAA3E02401FBE43A900173
:1079470023F0A3EBF090015AE0FAA3E0FB900129A2
:10795700EAF0A3EBF07962A3E3F009A3E3F0900167
:107967001DE0FF129849EE90012DF0A3EFF0900172
:1079770033E4F0A37404F0025F0D300303027B3C91
:10798700900132E0F5F090014DE065F07003027D63
:0179970017D8
:10799800900152E0B40001D34003E014F07F0712D5
:1079A8005078EE90017AF0A3EFF09001AE1201004A
:0979B80000000000E490014BF016
:1079C10090014BE025E0246CF582E43401F583E07D
:1079D100FCA3E0FD90014BE0FA2AFF246AF582E462
:1079E1003401F583ECF0A3EDF09001AE120089EFC4
:1079F100246AF582E43401F583E0FEA3E0FFE4FCB0
:107A0100FD1201289001AE1200D090014BE004F06C
:107A1100B408AD75F0039001AE1200C412000E90CF
:107A21000154EEF0A3EFF0A3E0FEA3E0FFE4FCFDC0
:107A3100121491C004C005C006C0077C0A7DD77E20
:107A4100A37F3C12112C121495EE900166F0A3EF66
:107A5100F0900154E0FCA3E0FDA3E0FAA3E0FB9069
:107A61000167E0F8EBC398FB900166E0F8EA98FA49
:107A7100F5F0ECB5F004EDB50300401EE0FAA3E02B
:107A8100FB900157E02BFB900156E03AFAF5F0EC40
:0A7A9100B5F005EDB50301D3401573
:107A9B00900156E0FEA3E0FF7D0712493EEE9001F8
:107AAB0054F0A3EFF01207CFEE90018EF0A3EFF09E
:0F7ABB009001AE12010000000000E490014BF0BA
:107ACA0090014BE025E02480F582E43401F583E05F
:107ADA00FCA3E0FD90014BE0FA2AFF247EF582E444
:107AEA003401F583ECF0A3EDF09001AE120089EFBA
:107AFA00247EF582E43401F583E0FEA3E0FFE4FC92
:107B0A00FD1201289001AE1200D090014BE004F062
:107B1A00B408AD75F0039001AE1200C412000E90C5
:107B2A00015AEEF0A3EFF0900132E090014DF0021D
:027B3A007D17B5
:107B3C00900132E0F5F090014DE065F07003027DAC
:017B4C001721
:107B4D00900152E0B40001D34003E014F01207CFCE
:107B5D00EE90018EF0A3EFF09001AE120100000047
:077B6D000000E490014BF061
:107B740090014BE025E02480F582E43401F583E0B4
:107B8400FEA3E0FF90014BE0FA2AFD7C00247EF581
:107B940082E43401F583EEF0A3EFF09001AE12001D
:107BA40089ED247EF582E43401F583E0FEA3E0FF51
:107BB400E4FD1201289001AE1200D090014BE004C4
:107BC400F0B408AC75F0039001AE1200C412000EBC
:107BD40090015AEEF0A3EFF09000DEE0B4052EE43D
:107BE400FCFD900158E0FEA3E0FF121491C004C014
:107BF40005C006C0077C0A7DD77EA37F3C12112CEA
:107C0400121495EE900166F0A3EFF0801C900141F0
:107C14001200897C0A7DD77EA37F3B12112C12149B
:107C240095EE900166F0A3EFF090015AE0FCA3E01A
:107C3400FD900158E0FAA3E0FB900167E0F8EBC384
:107C440098FB900166E0F8EA98FAF5F0ECB5F004D8
:107C5400EDB50300401EE0FAA3E0FB900159E02BD0
:107C6400FB900158E03AFAF5F0ECB5F005EDB503F8
:047C740001D34013E5
:107C7800900158E0FEA3E0FF124EC5EE90015AF0C5
:107C8800A3EFF07F07125078EE90017AF0A3EFF09F
:0F7C98009001AE12010000000000E490014BF0DB
:107CA70090014BE025E0246CF582E43401F583E094
:107CB700FEA3E0FF90014BE0FA2AFD7C00246AF561
:107CC70082E43401F583EEF0A3EFF09001AE1200E9
:107CD70089ED246AF582E43401F583E0FEA3E0FF31
:107CE700E4FD1201289001AE1200D090014BE00490
:107CF700F0B408AC75F0039001AE1200C412000E88
:107D0700900154EEF0A3EFF0900132E090014DF0B6
:107D17009000DEE06009E0B401028003027DDA90A2
:107D2700015EE0FAF5F0A3E0FB900154E0B5F00640
:0B7D3700A3E0B50301D34003027DDA96
:0F7D4200900147E004F0B40201D35003027DDF4B
:107D51007F05129849EE900129F0A3EFF01251F33B
:107D610075FD7F75ED7F75DD42D2DE1291EE7401F6
:107D710090010BF0C201E4900149F0740A90014FA7
:107D8100F0E4900151F07404900150F09000D6E0BD
:107D9100FAA3E0FB900121EAF0A3EBF0900135E0BA
:107DA100FAA3E02401FBE43A900123F0A3EBF0797C
:107DB1006290012BE3F009A3E3F090011DE0FF12B3
:107DC1009849EE90012DF0A3EFF0900133E4F0A378
:097DD1007404F01251F3025F0D7D
:107DDA00E4900147F09000DEE0FAB40101D35003C9
:107DEA00027ECB90015EE0FCA3E0FD900154E0B579
:107DFA000406A3E0B50501D34003027ECB90015AE5
:107E0A00E0FEA3E0FF900168E0FCA3E0FD900159C9
:107E1A00E02DFD900158E03CFCF5F0EEB5F005EFE1
:097E2A00B50501D35003027ECB23
:0F7E3300900148E004F0B40201D35003027ED066
:107E42007F05129849EE900129F0A3EFF01251F349
:107E520075FD7F75ED7F75DD42D2DE1291EE740104
:107E620090010BF0C201E4900149F0740A90014FB5
:107E7200F0E4900151F07404900150F09000D6E0CB
:107E8200FAA3E0FB900121EAF0A3EBF0900135E0C8
:107E9200FAA3E02401FBE43A900123F0A3EBF0798A
:107EA2006290012BE3F009A3E3F090011DE0FF12C1
:107EB2009849EE90012DF0A3EFF0900133E4F0A386
:097EC2007404F01251F3025F0D8B
:107ECB00E4900148F09000DEE06009E0B40102802C
:107EDB0003027F8E900113E0B40706A3E0B46C019C
:067EEB00D34003027F8E6C
:107EF100900162E0FAA3E0FB90015AE0B50206A30B
:0A7F0100E0B50301D35003027F89AD
:0C7F0B0090014AE004F0B40401D3407778
:107F17007F05129849EE900129F0A3EFF01251F373
:107F27001291EEE4900149F0740A90014FF0E49049
:107F37000151F07403900150F09000D6E0FAA3E0ED
:107F4700FB900121EAF0A3EBF0900135E0FAA3E002
:107F57002401FBE43A900123F0A3EBF0796290014E
:107F67002BE3F009A3E3F090011DE0FF129849EE1F
:107F770090012DF0A3EFF0900133E4F0A37404F027
:027F8700800573
:0E7F8900E490014AF09000DEE060030280EA1E
:107F970090015AE0FEA3E0FF900164E0FCA3E0FD3E
:107FA700900145E0FB1292E8EF640160030280EA6A
:0A7FB70090010BE0B40101D3407CFF
:107FC100E014F0740290014FF01251F3900125E496
:107FD100F0A3F0A3F0A3F09000D6E0FAA3E0FB90A9
:107FE1000121EAF0A3EBF0900135E0FAA3E02401CE
:107FF100FBE43A900123F0A3EBF090015AE0FAA3DD
:10800100E0FB900129EAF0A3EBF07962A3E3F00928
:10801100A3E3F090011DE0FF129849EE90012DF0CD
:10802100A3EFF090010DE0FBE4900133F0A3EBF03E
:10803100A3E4F0A3F0900132F0025F0D1251F3902E
:06804100011BE0B4013652
:108047001291EE75FE0175EE0175DE42D2DE9001EA
:1080570033740EF0A37410F0740990014FF090017F
:10806700ACE0FEA3E0FF7D0812493EEE900154F01C
:10807700A3EFF0025F0D1291EE7401900149F074C5
:108087000A90014FF0E4900151F0900150F09000F8
:10809700D6E0FAA3E0FB900121EAF0A3EBF0900110
:1080A70035E0FAA3E02401FBE43A900123F0A3EBC7
:1080B700F090015AE0FAA3E0FB900129EAF0A3EB64
:1080C700F07962A3E3F009A3E3F090011DE0FF124A
:1080D7009849EE90012DF0A3EFF0900133E4F0A35F
:0F80E7007404F09000DEE0B40102800302829581
:1080F60090015AE0FAF5F0A3E0FB7962E3B5F005EA
:1081060009E3B5030050077962EAF309EBF390013E
:108116005AE0FEA3E0FF12935BEF900150F0BF0020
:0781260001D34028200225CF
:10812D00900133E4F0A37478F0D202900150E0B4E2
:10813D0001067402900149F0900150E0B4020674FA
:10814D0004900149F0900133E06003028295A3E0B1
:0B815D0060030282952002030282955D
:0A81680090010BE0B40101D3407C4C
:10817200E014F0740290014FF01251F3900125E4E3
:10818200F0A3F0A3F0A3F09000D6E0FAA3E0FB90F6
:108192000121EAF0A3EBF0900135E0FAA3E024011B
:1081A200FBE43A900123F0A3EBF090015AE0FAA32A
:1081B200E0FB900129EAF0A3EBF07962A3E3F00976
:1081C200A3E3F090011DE0FF129849EE90012DF01B
:1081D200A3EFF090010DE0FBE4900133F0A3EBF08C
:1081E200A3E4F0A3F0900132F0025F0D1251F3907C
:0681F200011BE0B40136A0
:1081F8001291EE75FE0175EE0175DE42D2DE900138
:1082080033740EF0A37410F0740990014FF09001CC
:10821800ACE0FEA3E0FF7D0812493EEE900154F069
:10822800A3EFF0025F0D1291EE740A90014FF0E493
:10823800900151F0900150F09000D6E0FAA3E0FBD5
:10824800900121EAF0A3EBF0900135E0FAA3E024D5
:1082580001FBE43A900123F0A3EBF090015AE0FA15
:10826800A3E0FB900129EAF0A3EBF07962A3E3F025
:1082780009A3E3F090011DE0FF129849EE90012D4B
:10828800F0A3EFF0900133E4F0A37404F09000DE63
:0A829800E0B40101D350030283B5E6
:1082A20090015AE0FAF5F0A3E0FB7962E3B5F0053C
:1082B20009E3B5030050077962EAF309EBF3900191
:1082C20058E0FAA3E0FBA3E0FCA3E0FDECB5020456
:0982D200EDB50300400720030490
:1082DB00D202D2032003030283B5900160E0FAA31C
:1082EB00E0FB900154E0B50205A3E0B503004003A9
:1082FB000283B590015EE0FAA3E0FB900154E0B578
:10830B000206A3E0B50301D350030283B590015AD3
:10831B00E0FCA3E0FD900168E0FAA3E0FB900159BB
:10832B00E02BFB900158E03AFAF5F0ECB5F004EDD8
:05833B00B503005075C0
:10834000740190010BF01251F31291EEE490014987
:10835000F0740A90014FF0E4900151F0900150F058
:108360009000D6E0FAA3E0FB900121EAF0A3EBF045
:10837000900135E0FAA3E02401FBE43A900123F0F8
:10838000A3EBF090015AE0FAA3E0FB900129EAF098
:10839000A3EBF07962A3E3F009A3E3F090011DE001
:1083A000FF129849EE90012DF0A3EFF0900133E415
:1083B000F0A37404F09001AE1201000000000090E0
:1083C000011DE0FF129849EE9001A2F0A3EFF0E446
:0483D00090014BF0DD
:1083D40090014BE025E02494F582E43401F583E038
:1083E400FEA3E0FF90014BE0FA2AFD7C002492F505
:1083F40082E43401F583EEF0A3EFF09001AE1200B5
:1084040089ED2492F582E43401F583E0FEA3E0FFD4
:10841400E4FD1201289001AE1200D090014BE0045B
:10842400F0B408AC75F0039001AE1200C412000E53
:108434009001A8EEF0A3EFF090015CE0F5F0A3E06A
:10844400FB9001A8E0B5F005A3E0B50300400302EA
:0284540084DEC4
:0F845600900153E004F0B40401D350030284E317
:108465001251F31291EE740190010BF0E490014961
:10847500F0740A90014FF0E4900151F074059001F9
:1084850050F0900133E4F0A37404F09000D6E0FAC4
:10849500A3E0FB900121EAF0A3EBF0900135E0FAAF
:1084A500A3E02401FBE43A900123F0A3EBF0900153
:1084B5005AE0FAA3E0FB900129EAF0A3EBF0796218
:1084C500A3E3F009A3E3F09001A8E0FAA3E0FB9091
:0984D500012DEAF0A3EBF0800593
:1084DE00E4900153F09000D6E0C0E0A3E0C0E07B52
:1084EE00027A0079E17D057C5578C512081D15814B
:1084FE00158190010BE06401600A9000DEE0B4018A
:04850E0001D3401045
:108512007B027A0079E39000DEE0FD128F8E8017F5
:1085220074439000E4F004A3F0743AA3F090010BBA
:0A853200E024309000E7F020020A78
:0A853C0090012FE09000E1F0800DA7
:10854600900130E0B4010674049000E1F0740590E7
:1085560000E2F07F017B027A0079E1129138900106
:0785660052E060030286727F
:10856D00900135E060030285F6A3E0707C90013246
:10857D00E0FBE4C0E0C003FCFD900154E0FEA3E08D
:10858D00FF121491C004C005C006C0079001391236
:10859D001285C004C005C006C0077C6F7D127E83A6
:1085AD007F3A12112CC004C005C006C00790015AB5
:1085BD00E0FEA3E0FFE4FCFD121491C004C005C071
:1085CD0006C007900141121285C004C005C006C047
:1085DD00077B027A0079E17D057C5578D612081D5E
:1085ED0074F62581F5810286C8900135E0C0E0A3BF
:1085FD00E0C0E0E4FCFD900154E0FEA3E0FF1214A6
:10860D0091C004C005C006C007900139121285C083
:10861D0004C005C006C0077C6F7D127E837F3A12B1
:10862D00112CC004C005C006C00790015AE0FEA37E
:10863D00E0FFE4FCFD121491C004C005C006C007A4
:10864D00900141121285C004C005C006C0077B020F
:10865D007A0079E17D057C5578E912081D74F625BF
:05866D0081F58180563B
:10867200E5FEFF7E00E4FC7D6412013DE4FC7DFF2B
:10868200120151C006C007E4FCFD9001A8E0FEA360
:10869200E0FF121491C004C005C006C0079001415A
:1086A200121285C004C005C006C0077B027A007999
:1086B200E17D057C5578FC12081D74FA2581F5814F
:1086C20074259000F0F07F027B027A0079E112912A
:0E86D20038025F0D9000D8E0705DA3E0705993
:1086E0009000D7E004F09000D67003E004F0E4C0FE
:1086F000E0C0E07461C0E07445C0E0E4FCFD9001BE
:1087000054E0FEA3E0FF121491C004C005C006C0EF
:1087100007900139121285121288C004C005C006E4
:10872000C007E4FCFD74C8FE7442FF12112C121441
:1087300095EE9000D8F0A3EFF090014CE0B4020267
:0587400080030287CA5E
:0E8745007B057A56790E128E97EF64017077DD
:108753001251F31291EE740190010BF0E490014970
:10876300F0740A90014FF0E4900151F0740290010B
:1087730050F09000D6E0FAA3E0FB900121EAF0A3C9
:10878300EBF0900135E0FAA3E0FB900123EAF0A3BC
:10879300EBF090015AE0FAA3E0FB900129EAF0A381
:1087A300EBF07962A3E3F009A3E3F090011DE0FF8E
:1087B300129849EE90012DF0A3EFF0900133E4F00D
:1087C300A37404F0025F0D900133E0FAA3E0BA0052
:0A87D30004B40001D35003028A39F8
:1087DD00900132E0F5F090014DE065F07003028AF2
:0187ED009DEE
:1087EE00B2B39001ACE0FEA3E0FF7D0712493EEE6E
:1087FE00900154F0A3EFF01207CFEE90015AF0A3C0
:10880E00EFF09000D6E0C0E0A3E0C0E07B027A007B
:10881E0079E17D057C56788412081D1581158174C9
:10882E00069000E1F07F017B027A0079E112913827
:10883E00E4FCFD900154E0FEA3E0FF121491C0048D
:10884E00C005C006C007900139121285C004C005CC
:10885E00C006C007E4FCFD74C8FE7442FF12152268
:10886E00BF017C900135E0C0E0A3E0C0E0E4FCFD78
:10887E00900154E0FEA3E0FF121491C004C005C0A5
:10888E0006C007900139121285C004C005C006C08B
:10889E00077C6F7D127E837F3A12112CC004C005B7
:1088AE00C006C00790015AE0FEA3E0FFE4FCFD12F3
:1088BE001491C004C005C006C00790014112128574
:1088CE00C004C005C006C0077B027A0079E17D05B1
:0F88DE007C5578E912081D74F62581F5818071AB
:1088ED00E4FCFD900154E0FEA3E0FF121491C004DE
:1088FD00C005C006C007900139121285121495EFFC
:10890D00900146F0900135E0C0E0A3E0C0E0900199
:10891D0046E0FBE4C0E0C00390015AE0FEA3E0FF97
:10892D00E4FCFD121491C004C005C006C0079001FF
:10893D0041121285C004C005C006C0077B027A0033
:10894D0079E17D057C56789512081D74F82581F521
:10895D00817F027B027A0079E1129138900132E039
:10896D0090014DF09000DEE06009E0B4010280035B
:10897D00028A3190015EE0FAF5F0A3E0FB9001541C
:0F898D00E0B5F006A3E0B50301D34003028A3141
:0F899C00900147E004F0B40301D35003028A3680
:1089AB007F05129849EE900129F0A3EFF01251F3D5
:1089BB0075FD7F75ED7F75DD42D2DE1291EE740190
:1089CB0090010BF0C201E4900149F0740A90014F41
:1089DB00F0E4900151F07404900150F09000D6E057
:1089EB00FAA3E0FB900121EAF0A3EBF0900135E054
:1089FB00FAA3E0FB900123EAF0A3EBF0796290017C
:108A0B002BE3F009A3E3F090011DE0FF129849EE70
:108A1B0090012DF0A3EFF0900133E4F0A37404F078
:068A2B001251F3025F0D81
:088A3100E4900147F0028D5FA3
:108A39001291EE740A90014FF0E4900151F0900107
:108A490050F09000D6E0FAA3E0FB900121EAF0A3F0
:108A5900EBF0900135E0FAA3E0FB900123EAF0A3E3
:108A6900EBF090015AE0FAA3E0FB900129EAF0A3A8
:108A7900EBF07962A3E3F009A3E3F090011DE0FFB5
:108A8900129849EE90012DF0A3EFF0900133E4F034
:108A9900A37404F0025F0DD2B2D2B3900150E0B4D6
:108AA90003028050500BE06012146022146032807F
:0B8AB9007AE024FC60511460618070C2
:108AC4007B027A0079E17D057C5678A712081DD2D5
:108AD400B4805D7B027A0079E17D057C5678B8121A
:108AE400081DD2B4804A7B027A0079E17D057C5668
:108AF40078C912081DC2B480377B027A0079E17DFF
:108B0400057C5678DA12081DC2B480247B027A00F0
:108B140079E17D057C5678EB12081DC2B480117B87
:108B2400027A0079E17D057C5678FC12081DC2B4F6
:108B340074069000E1F07F017B027A0079E11291E2
:108B440038900133E0FAA3E0FBBA0004B40401D383
:108B54004009900133E4F0A37404F0900133E07011
:058B64001EA3E0701AE1
:108B690012919A900133E4F0A37404F0900151E05A
:108B790004F0B40601D34002E4F0900151E0B403DB
:108B890003028C1D500CE0602014604814606502DB
:108B99008D44E024FC7003028C3D147003028CACFC
:098BA900147003028D0B028D44CF
:108BB200900126E0F4FB900125E0F4FA0BEB700142
:108BC2000AC002C0037B027A0079E17D057C5778F6
:108BD2000D12081D15811581028D44900127E0C0F8
:108BE200E0A3E0C0E07B027A0079E17D057C577862
:108BF2001E12081D15811581028D44900121E0C0CD
:108C0200E0A3E0C0E07B027A0079E17D057C577841
:108C12002F12081D15811581028D44900123E0C099
:108C2200E0A3E0C0E07B027A0079E17D057C577821
:108C32004012081D15811581028D44900149E060A2
:108C42000F14601E14602D14603C14604B028D449E
:108C52007B027A0079E17D057C57785112081D026A
:108C62008D447B027A0079E17D057C577862120897
:108C72001D028D447B027A0079E17D057C57787371
:108C820012081D028D447B027A0079E17D057C5732
:108C9200788412081D028D447B027A0079E17D05F9
:108CA2007C57789512081D028D44E4FCFD90012941
:108CB200E0FEA3E0FF121491C004C005C006C00785
:108CC200900141121285C004C005C006C007E4FC31
:108CD200FD90012BE0FEA3E0FF121491C004C00539
:108CE200C006C007900141121285C004C005C0062B
:108CF200C0077B027A0079E17D057C5778A61208CD
:108D02001D74F82581F5818039E4FCFD90012DE088
:108D1200FEA3E0FF121491C004C005C006C0079074
:108D22000141121285C004C005C006C0077B027A49
:108D32000079E17D057C5778B812081D74FC258105
:108D4200F5817F027B027A0079E112913890014C21
:048D5200E0B402097E
:0C8D56001207F5740190014FF0025F0D50
:108D6200900116E0B401004007E0B40301D34006CD
:108D72007401900116F090011DE0B40401D3400388
:108D82007404F0900113E0FAA3E0FBBA0603B440C6
:108D9200004009BA0704BB6C01D3400A9001137466
:108DA20007F0A37476F0900109E0FAA3E0FBBA01A0
:108DB20003B4F4004009BA0904BBC401D3400A90C9
:108DC20001097404F0A374B0F090011EE0FAA3E06C
:108DD200FBBA0703B4D0004009BA0B04BBB801D3F5
:108DE200400A90011E7408F0A37484F0900110E010
:108DF200FAA3E0FBBA0103B4F4004009BA0404BBCD
:108E0200B001D3400A9001107403F0A374E8F0900B
:108E12000117E0B405004007E0B41901D34006741D
:108E22000F900117F0900120E0B40101D3400374C8
:108E320001F090011AE0B41E00400AE0FB7A00B48F
:108E4200F001D34006743C90011AF090010DE0B499
:108E52001E00400AE0FB7A00B4F001D34006743CE5
:108E620090010DF090010EE0FAA3E0FBBA0103B409
:108E7200F4004009BA0904BBC401D3400A90010EB0
:108E82007404F0A374B0F0900118E0B40101D3406F
:058E9200037401F02251
:108E97007841EBF208EAF208E9F21207F574199043
:108EA70001B2F0900130E024FF92047F017941E3A1
:108EB700C0E009E3C0E009E3F9D002D0031291381A
:108EC7007B027A0079E17D057C5778CA12081D7408
:108ED700069000E3F0E49001B3F0A3F09001B4E052
:078EE70064027003028F70AA
:108EEE00900120E0B40103120003129201EF9001F1
:0A8EFE00B4F064016004E0B403293D
:078F08009001B3E0B4011079
:108F0F00E4F074069000E3F074209000EAF0801211
:108F1F0074019001B3F074209000E3F07406900098
:108F2F00EAF07F027B027A0079E1129138900130EA
:108F3F00E0B4010874079000F0F0800674209000F0
:0E8F4F00F0F0A204E433FA900130E06A60868C
:108F5D00E024FF92049001B2E014F06003028EE36E
:098F6D00E4FF229001B3E0FF22B1
:108F76004E6943444E694D484C6946654C69496F94
:088F86004C69506F534C41206F
:108F8E007844EBF208EAF208E9F28D07E49001B5B5
:018F9E00F0E2
:108F9F00EF25E025E0FE9001B5E02E908F7693FE51
:108FAF007944E3FD09E3FC09E3F8EE120026794664
:108FBF00E304F3197003E304F39001B5E004F0B494
:038FCF0004CE22AB
:108FD200900121E4F0A3F0A3F0A3F0A3F0A3F0A387
:108FE200F0A3F0A3F0A3F0A3F0A3F0A3F0A3F02268
:0B8FF200EEB40005EFB40001D340070F
:088FFD00EF1F70F11E80EE224F
:10900500C283E4FE7F64128FF27F3312906F7F324A
:1090150012906F7F2812906F7F0C12906F7F06124F
:0F902500906F7F0112906F7E017FF4128FF22205
:109034008F0553800FED54F04280D283E4FE7F32DB
:10904400128FF2C28353800FEDC454F04280D28356
:10905400E4FE7F32128FF2C2837E017FF4128FF21C
:0190640022E9
:0A9065007847EFF2D2821290342215
:0A906F007848EFF2C282129034221A
:109079000E1F111111111F000E1F1111111F1F00B9
:109089000E1F11111F1F1F000E1F111F1F1F1F0071
:109099000E1F1F1F1F1F1F000002060E06020000E1
:1090A90000080C0E0C080000001F1517111F000006
:1090B900001F10101010101F001F00000000001FDB
:1090C900001F01010101011F001F1F1F1F1F1F1F7B
:1090D9000E1F11111F1F1F000002060E06020000BD
:1090E90000080C0E0C080000001F1517111F0000C6
:1090F9007849EFF27440794AF37949E375F040A46D
:079109007949F3E4794BF30F
:10911000794AE3FF12906F7949E3FA784BE22A909B
:10912000907993FF129065794AE304F3794BE30455
:08913000F3794BE3B440D922AE
:10913800784CEFF2784DEBF208EAF208E9F2EF1416
:0C914800600A14600E14601214601622FD
:109154007F8012906F80137FC012906F800C7FFF0E
:0E91640012906F80057FFF12906FE47950F338
:10917200794DE3FD09E3FC09E3F812005EFF12906A
:1091820065794FE304F3197003E304F37950E304C0
:08919200F37950E3B410D92277
:07919A0090011CE0B401216B
:0491A100E47953F327
:1091A500C2B5E4FE7F281291D6D2B5E4FE7F3C120B
:0E91B50091D67953E304F37953E3B406E32231
:0791C30090011CE0B4010B58
:0C91CA00C2B5E4FE7F3C1291D6D2B52263
:0491D600EE4F6013E5
:1091DA007B007A06DBFEDAFC7C06E4FDEF1F70EC0E
:0491EA001E80E922D8
:0791EE0090011CE0B4010B2D
:0C91F500C2B57E037F201291D6D2B522B5
:10920100E47955F3208004047955F3208105740233
:109211007955F320800820810574037955F3795538
:0C922100E360031291C330800320812918
:10922D00E4FE7F321291D67954E3B40F01D340128C
:06923D007955E3B40207BD
:10924300E47954F37F04227955E3FF227954E3044C
:0C925300F380D1E47954F37955E3FF2255
:0B925F007951E39001B6F0C205FF2238
:0F926A002006FDEF7952F3D206300702D2992287
:109279007856EBF208EAF208E9F27956E3FD09E3D8
:0B928900FC09E3F812005E6424602181
:109294001200037956E3FD09E3FC09E3F812005ECA
:1092A400FF12926A7958E304F31970D3E304F3804C
:0292B400CE22C8
:0A92B600C0E0C0D0E9C00130980DFF
:0D92C000C298E5997951F3D205C298801447
:0392CD0030060D5B
:0D92D000C2067952E3F599C299C2078004E5
:0B92DD00C299D207D001D0D0D0E032FF
:1092E8007878EEF208EFF2787AECF208EDF2787C12
:1092F800EBF27962E38EF0B5F00709E38FF0B5F091
:0393080000500D05
:0D930B00E4797DF37962EEF309EFF3804021
:109318007879E2FF7963E3C39FFF18E2FB19E39BC7
:10932800FE12020EEF797DF3797CE3F5F0787DE2A9
:10933800B5F001D3401A787AE2F5F07978E3B5F020
:109348000A08E2F5F009E3B5F001D340037F0122F2
:03935800E4FF220D
:10935B00787EEEF208EFF2900135E0FAA3E0FB79AC
:10936B0059E3FD7C00E4B502098BF0ED6B70030251
:0E937B0094FCBA0004BB0001D350030294FC22
:10938900EB7959F31294FF900135E0FAA3E0BA00A2
:0693990003B40600501EA3
:04939F00E47980F3FA
:1093A3007980E3FA2A246EF8E4F208F27980E30480
:0F93B300F37980E3B405E9E4FF2274057980F3D0
:1093C2007980E3FB25E0246AF8EB25E0246CF9E2DE
:1093D200F30809E2F37980E314F37980E3B400013E
:1093E200D350DD129553EE796EF309EFF390011825
:0793F200E0B40001D34000CC
:0E93F900900135E0B40005A3E0B40A00501066
:10940700795EE4F3097463F3795CE4FFF309F3220B
:0C941700795AE4F3097463F3E47980F3FC
:109423007880E2FA2A246EF8795AE3F5F0E2B5F08F
:0C9433000909E3F5F008E2B5F000500D67
:10943F00EA2A246EF8795AE2F30809E2F37980E315
:10944F0004F37980E3B405CC900118E0B40001D3A4
:02945F004000CB
:10946100795EE3701909E37015785CE2701008E227
:0B947100700C785AE2700708E27003EC
:10947C007F0222795EE3F5F0785AE2B5F00909E350
:09948C00F5F008E2B5F000501201
:10949500795A785EE3F20908E3F2795CE4FFF309AF
:0B94A500F322795CE3701109E3700D05
:1094B000796E785CE3F20908E3F2E4FF22795CE379
:1094C000F5F0786EE2B5F00909E3F5F008E2B5F0E1
:0394D00000400D4C
:1094D300796E785CE3F20908E3F2E4FF22785FE255
:1094E300FA795DE3C39AFB18E2FC19E39CB4000428
:0694F300BB0201D340039F
:0694F9007F0122E4FF22C6
:1094FF007881EEF208EFF27960E3700C09E37008FF
:0A950F007960EEF309EFF3227F0507
:10951900EF25E02460F8EF25E02462F9E2F3080979
:10952900E2F3DFEC7861E2FA7982E3C39AFF18E2A9
:10953900FB19E39BFE12020EEE7964F309EFF3794E
:0A954900817860E3F20908E3F222E2
:109553007967E3FB19E3FAEBC333CA33CAFB7965D3
:10956300E32BFB19E33AFA7968E3FC09E3FDE4FE34
:109573007F0312013DEB2FFFEA3EFE786BE2FB18FF
:10958300E2FAEBC333CA33CAFBEF2BFBEE3AFA78AA
:109593006DE22BFF18E23AFEE4FCFD121491C004C5
:1095A300C005C006C0077C397D8E7EE37F3D121166
:1095B3002C121495EE7883F208EFF218E2FE08E21B
:0295C300FF2285
:0995C500C2A3C2A2D2A1D2A022CD
:1095CE007885ECF208EDF29001B77403F0A374E81D
:1095DE00F0D2A3EF2400FBEE34057987F309EBF309
:1095EE0019E3FE09E3FF12972F7985E3FE09E3FFE6
:0995FE0012978E1297EBC2A32212
:109607009001B77401F0A3742CF0D2A3EF2400FBF0
:10961700EE34067989F309EBF319E3FE09E3FF1248
:10962700972F12963CEE798BF309EFF3C2A319E358
:05963700FE09E3FF2223
:10963C00798DE4F309F3798FF309740FF3798FE3E0
:07964C006480B48000403D82
:10965300129815A2A0E4335401FBE47991F309EBCA
:10966300F37890E2FAE3FD19E3FC0AED8005C333D6
:10967300CC33CCDAF9FD798EE34DF319E34CF3796E
:1096830090E314F3F41970BEE314F380B9798DE316
:05969300FE09E3FF22C7
:109698009001B77403F0A374E8F0D2A37E047FC0EE
:0696A80012972FC2A3225D
:1096AE009001B77403F0A374E8F0D2A37E047F8018
:0996BE0012972F1297EBC2A322B0
:1096C7007893EEF208EFF29001B77403F0A374E811
:1096D700F0D2A37E047F4012972F7993E3FE09E32C
:0A96E700FF12978E1297EBC2A32228
:1096F1009001B77403F0A374E8F0D2A3EF2400FB48
:10970100EE34077995F309EBF319E3FE09E3FF1250
:08971100972F1297EBC2A3226F
:109719009001B77403F0A374E8F0D2A37E04E4FFC8
:0697290012972FC2A322DB
:10972F007897EEF208EFF27999E4F309740AF37976
:09973F0099E36480B4800040430A
:10974800789AE2FA7998E3FD19E3FC0A8005C313D5
:10975800CD13CDDAF9ED5401FD7C00E4799BF309D2
:10976800EDF319E3B4000909E3B40104D2A18002BE
:10977800C2A1129815799AE314F3F41970B8E31496
:06978800F380B3C2A12230
:10978E00789DEEF208EFF2799FE4F309740FF37906
:09979E009FE36480B480004043A5
:1097A70078A0E2FA799EE3FD19E3FC0A8005C3136A
:1097B700CD13CDDAF9ED5401FD7C00E479A1F3096D
:1097C700EDF319E3B4000909E3B40104D2A180025F
:1097D700C2A112981579A0E314F3F41970B8E31431
:0497E700F380B32236
:1097EB00C2A39001B7E0FEA3E0FF129830D2A3749E
:1097FB00FFFAFB20A013EA6480B48004BB0001D302
:0A980B004007EB1B70ED1A80EA2203
:10981500D2A29001B7E0FEA3E0FF129830C2A29059
:0B98250001B7E0FEA3E0FF1298302224
:10983000E4FAFB8EF0EAB5F0068FF0EBB5F00050DD
:09984000070BEB70EE0A80EB222D
:1098490078A3EFF29001BA12010000000000E49041
:0398590001B9F062
:10985C00E4FE7FC8128FF279A3E3FF1298B1EE9069
:10986C0001BEF0A3EFF09001BA120089E4FCFD9068
:10987C0001BEE0FEA3E0FF1201289001BA1200D055
:10988C009001B9E004F0648070C675F007A3120073
:10989C00C412000E9001BEEEF0A3EFF09001BEE0FA
:0598AC00FEA3E0FF2215
:1098B100EF441823232354F8FFD2A40000D2A700B9
:0798C10000C2A700007E05B4
:1098C800C2A4EF30E704D2A68002C2A6EFC333FFDA
:1098D8000000D2A40000DEE8D2A6C2A40000D2A4F0
:0A98E8000000C2A400007F007E050E
:1098F200EFC333FF30A5034401FFD2A40000C2A48A
:0E9902000000DEECEF540FFC7D007F007E08BD
:10991000EFC333FF30A5034401FFD2A40000C2A46B
:0D9920000000DEECEF2DFFE43CFED2A7229C
:00000001FF
